:100000000C94BF270C9435280C9435280C94352873
:100010000C9435280C9435280C9435280C943528EC
:100020000C9435280C9435280C9435280C943528DC
:100030000C9435280C9491280C94D0280C943528D5
:100040000C9435280C9435280C9435280C943528BC
:100050000C9435280C9435280C9435280C943528AC
:100060000C9435280C9435280C9435280C9435289C
:100070005A5501200101003808000000000000006E
:100080000000000000000000000000000000000070
:10009000810045005DFF5E1027FF2AD22B7D210CD9
:1000A00022FB850084008903888D81096F02444208
:1000B00047004501B083B300B10124B925578A1D1B
:1000C0008B03832B862B8F2B942B9C2BA52BAA2B5E
:1000D000AF2BB22BC42BC72BCA2B0B2C0E2C112CE5
:1000E00000020800085504085A0000F800099000B2
:1000F0000A1E32050000FF000000E00000000000C2
:1001000000000000000000000000000000000000EF
:1001100000000000000000000000000000000000DF
:1001200000000000000000000000000000000000CF
:1001300000000000000000000000000000000000BF
:1001400000000000000000000000000000000000AF
:1001500000000049000000495252000052525C2D3C
:10016000000000000000000000000000000000008F
:100170000040000000494A52004952525B1C525351
:100180001C25241B2425251B0A0A2D1C12120A0AD1
:100190000000000000000000404949494949525B05
:1001A0005B5B525B1C1C1312241C12090909120907
:1001B0000909090A0A0A0A0A0A13120A0A12130A80
:1001C00000000000000092525252525213121309C2
:1001D000001C0A1212401B65090A0009241B1200A8
:1001E00000251C1C010025241C1C0024252424247B
:1001F0000000000000005249494000001B13524912
:100200004900641C1C5B4A481C651C2552491C1C87
:10021000652464491C1C652564491C1C6D2E5C49C1
:100220000000000000000000000000490000000085
:10023000535200000053522500004A522525000069
:100240005B251300005B53000A1C095B1C657F37AC
:100250004052522E2E1C525C2E251B1324251C1C92
:1002600012002525120000121B0000132E37001B60
:1002700037372E2E37372E2E2E2E2E2E6E6E6E1CCC
:100280001313120009131200001213130012251C7D
:1002900013132E371C131313361C131B1B1B251390
:1002A0001C1C1B1B1B1C1C1C1C1C1C1C1C1C1C139A
:1002B0001312121313001313131C000913131C0140
:1002C0000037131C13002E2E1C1C001C772E25003B
:1002D000137F251C010A37241C1C0A2E2525090022
:1002E000132E242525252E252525252525252D2EAE
:1002F000251B2E2E251C1325251C1C1C1C011C1C1B
:100300001300011C0A000165775C016E7F6E521BB1
:1003100025256D1C524925251C1353001C1C1C52FD
:100320004A001B135B5B000009525C0000005B5C31
:10033000000000001B0000000000000000000000A2
:10034000135B7F776E6E136577766E6E1B657776BF
:1003500076761B5BBF76B67609136DBFB7B6001B0A
:10036000125C76BF0000121B125B00000000090A3D
:100370006E6E6E77241C6E6E77251C1C6E776E1C5D
:100380001C1C76761C1C2425B765646D6D1B766D70
:100390006D5B09125B5C5B125B641213131B121220
:1003A0001C1C1C1C1C241C1C242525242425251B4A
:1003B00000002513000064BF00096EBFBF6D6EBF53
:1003C0006D5B12135B12131209000901000000009B
:1003D0002E1C0900096E010009767F7F12777F7F4E
:1003E0006412BF775B121B095B121B0900001B091B
:1003F00000000000000000000000000000000000FD
:100400007F7F5313130064121B0100001B120000B6
:1004100000000000000000000000000000000000DC
:1004200000000000000000000000000000000000CC
:100430000000000000002600000026002F00000041
:100440002F00370000003700FF000000FF00BF0052
:100450000000BF0037000037000000262600000023
:1004600000000000000026262626260000000000CE
:100470002F000000003700000000FF00000000BF58
:100480000000000037000000000026262626260077
:100490000000000000002626262626002F0000006F
:1004A0000000370000000000FFFFFFFF0000BF005A
:1004B0000000000037000000000026262626260047
:1004C0000000000000002626262600002F00000065
:1004D0002F00370000003700FFFFFFFF0000BF00C4
:1004E0000000BF0037000000370026262626000047
:1004F000000000000000000026262600002F00005B
:100500002F00370000003700FF000000FF00BF0091
:100510000000BF003700003700002626260000003C
:100520000000000000002600000026002F00000050
:100530002F000037003700000000FF00000000BF60
:1005400000BF000037000000370026000000260032
:10055000000000000000000000000000000000009B
:10056000000000000000000000000000000000008B
:100570000000009B000000529BA400005B9B6D7775
:10058000000000000000000000000000000000006B
:10059000005B000000E4F6FF099BEDF6FFBFA4AD91
:1005A000BFBFBFBF767F7FB7B7BF7F766EB7B7BF1E
:1005B00000000000000000005BB6F6F6F6FFFFFF4B
:1005C000FFBFFFFFFFBFBFAEFFFFFFB7AD65FFFF80
:1005D000B7B6AD65FFFFBFB7AE6EFFFFBFB7B7657C
:1005E000000000000000F6F6EDEDADA4B66D6D5C08
:1005F000526E6565655265765C5C52536E24655239
:10060000526E25255B52772D2525526E6E2D2525A0
:10061000000000000000A49B9B4900006564A49BAF
:1006200092006D2525649349656E652E9B522425A5
:100630006D25655225246D2D655225256E2E64523B
:1006400000000000000000000000004A0000000060
:100650005B9B0000005B5B2D0000525B2E2E0001B7
:100660005B2D1C01005C5B014A654A5B1C6E7F7759
:10067000495B9B77776D5B65776E65656D2D25258D
:100680005C522E25130949641C09095C7F7F091CF3
:100690007F7F777F777F77777F7F7776777F7F6EB4
:1006A000656E6EA4B6FF655BA4B7BFFF526DBFBF9A
:1006B000BFFF7FBFBFBFBFFFBFBFB7BFFFFF7FB7DA
:1006C000BFBFFFFF6EB7BFBFFFFF77BFBFBFFFFF5B
:1006D000FFFFBFBFB75BFFFFBFBFA464FFFFBFAD9E
:1006E000A47FFFFFBFA4BF7FFFBFADBFBFBFFFB6EB
:1006F000BFBFBF77F7BFBFBF7777FFBFBFBF645232
:100700006D7F6E2E2D2D7F766E6E6E2E77777776BF
:100710002E1C7F776E251C25776525251C096E6E9E
:100720001C0949255B494A6E7F645377BF775B5C40
:10073000256E6E255B4A25651C1B5B002524245B0A
:1007400053001C1B5B5C00000A5B640000006464D7
:10075000000000005C00000000000000000000003D
:100760005B5C7FBF77765C6D7FB777775C6D7FBFB3
:1007700077775C64BFBFBFBF0A5C6EBFBFBF006559
:10078000646DBFBF00005B6D646D00000000125B14
:100790007777777F6E6E77777F766D7677BF776DB9
:1007A0006E76BF7F6D6E767FBF7676BFBF76BFBF3A
:1007B000BFB664ADADB6B6ADBFFF646DADB6AD64EA
:1007C00077BFBFBFFFFF77BFBFBFFFFF7FBFBFBF09
:1007D000FFF6BFB7ADF6FFFFA4ADFFFFFFFFFFFFC2
:1007E000FFFFFFFFFFFFFFF6A4005B5200000000C9
:1007F000BFBFAD5B64BFB6ADADBFFFBFFFFFFFFFC7
:10080000BF64FFFFBFB6765BFFBFBF5B0000FF5C4E
:1008100000000000000000000000000000000000D8
:10082000BFBF645C5C006E5C654900006D5B0000EE
:1008300000000000000000000000000000000000B8
:1008400000000000000000000000000000000000A8
:10085000060004000000010002000300040005007F
:1008600006000700080009000A000B000C000D003C
:100870000E000F0010000000110012001300140001
:1008800015001600060003000000170018001900EC
:100890001A001B001C001D001E001F00200021006C
:1008A000220023002400250026000000004088913B
:1008B000D2E4ADB5B6BEBFFF444F574E00464945E2
:1008C0004C4420504F532E005941524453204C4524
:1008D00046540054494D4500484F4D450056495334
:1008E00049544F52002D4900492D002A2A2A2A2A0C
:1008F00020544F554348444F574E202A2A2A2A2A2B
:10090000002A2A20204348414E4745205349444568
:100910005320202A2A002A2034544820444F574E7E
:10092000204B49434B204F522052554E202A002A3B
:1009300020315354205155415254455220454E4484
:1009400053202A002A20324E44205155415254450A
:100950005220454E4453202A002A2033524420512D
:1009600055415254455220454E4453202A002A20D6
:10097000345448205155415254455220454E445319
:10098000202A0057494E53205749544800544F00DD
:1009900049542049532041204452415721212100EC
:1009A0003E3E2050524553532053544152542054FC
:1009B0004F2052455455524E20544F204D454E55D0
:1009C000203C3C003230323220444F4D494E494B9E
:1009D000204B52495354454E0053544152540053F6
:1009E0004F554E443A004C4556454C3A004F4E2028
:1009F000004F46460045415359004E4F524D004866
:100A0000415244000000000000000000000000000F
:100A100000000000000000000000000000000000D6
:100A200000000000000000000000000000000000C6
:100A3000000000000000FF00000000FFFFFF0000BA
:100A400000FFFFFF00000000FF0000000000FF00AB
:100A500000000000000000000000FF000000000097
:100A600000000000FFFF00FFFF00FFFF00FFFF008E
:100A7000FF0000FF00000000000000000000000078
:100A80000000000000000000000000000000000066
:100A90000000000000000000000000FF00FF000058
:100AA000FFFFFFFFFF0000FF00FF000000FF00FF4F
:100AB0000000FFFFFFFFFF0000FF00FF000000003D
:100AC0000000000000FF0000000000FFFFFF00002A
:100AD000FF000000000000FFFF000000000000FF1A
:100AE0000000FFFFFF0000000000FF00000000000A
:100AF00000000000FFFF0000FF00FFFF0000FF00FC
:100B0000000000FF00000000FF00000000FF0000E8
:100B10000000FF0000FFFF00FF0000FFFF000000DB
:100B20000000000000FF00000000FF00FF000000C8
:100B3000FF00FF00000000FF00000000FF00FF00BA
:100B4000FF00FF0000FF000000FFFF00FF000000AB
:100B50000000000000FFFF00000000FFFF00000099
:100B600000FF000000000000000000000000000086
:100B70000000000000000000000000000000000075
:100B8000000000000000FF00000000FF0000000067
:100B900000FF0000000000FF0000000000FF000058
:100BA000000000FF000000000000FF000000000047
:100BB0000000000000FF000000000000FF00000037
:100BC0000000FF0000000000FF0000000000FF0028
:100BD00000000000FF00000000FF00000000000017
:100BE0000000000000000000000000FF00FF000007
:100BF00000FFFFFF0000FFFFFFFFFF0000FFFFFF00
:100C0000000000FF00FF00000000000000000000E6
:100C1000000000000000000000000000FF000000D5
:100C20000000FF000000FFFFFFFFFF000000FF00CB
:100C300000000000FF0000000000000000000000B5
:100C400000000000000000000000000000000000A4
:100C50000000000000000000000000000000000094
:100C6000000000FFFF00000000FFFF00000000FF89
:100C70000000000000000000000000000000000074
:100C8000000000000000FFFFFFFFFF000000000069
:100C90000000000000000000000000000000000054
:100CA0000000000000000000000000000000000044
:100CB0000000000000000000000000000000000034
:100CC000000000FFFF00000000FFFF000000000028
:100CD0000000000000000000000000000000FF0015
:100CE000000000FF00000000FF00000000FF000007
:100CF0000000FF00000000000000000000000000F5
:100D000000000000002F2F2F00002F0000002F00F8
:100D10002F00002F2F002F002F002F002F2F00005B
:100D20002F002F0000002F00002F2F2F00000000A9
:100D30000000000000002F000000002F2F00000026
:100D400000002F00000000002F00000000002F0016
:100D5000000000002F000000002F2F2F00000000D7
:100D600000000000002F2F2F00002F0000002F0098
:100D7000000000002F0000002F2F0000002F0000B7
:100D800000002F00000000002F2F2F2F2F00000049
:100D900000000000002F2F2F00002F0000002F0068
:100DA000000000002F00002F2F2F00000000000087
:100DB0002F002F0000002F00002F2F2F0000000019
:100DC000000000000000002F000000002F2F000096
:100DD000002F002F00002F00002F00002F2F2F2F9B
:100DE0002F000000002F00000000002F0000000076
:100DF000000000002F2F2F2F2F002F0000000000D9
:100E00002F00000000002F2F2F2F000000000000F7
:100E10002F002F0000002F00002F2F2F00000000B8
:100E20000000000000002F2F0000002F0000000035
:100E30002F00000000002F2F2F2F00002F00000098
:100E40002F002F0000002F00002F2F2F0000000088
:100E5000000000002F2F2F2F2F00000000002F0078
:100E60000000002F000000002F000000002F0000F5
:100E70000000002F00000000002F00000000000014
:100E800000000000002F2F2F00002F0000002F0077
:100E90002F0000002F00002F2F2F00002F00000038
:100EA0002F002F0000002F00002F2F2F0000000028
:100EB00000000000002F2F2F00002F0000002F0047
:100EC0002F0000002F00002F2F2F2F000000000008
:100ED0002F000000002F0000002F2F000000000056
:100EE0000000000000000000000000000000000002
:100EF00000FFFF00000000FFFF00000000000000F6
:100F0000000000FFFF00000000FFFF0000000000E5
:100F100000000000000000000000000000000000D1
:100F200000FFFF00000000FFFF00000000000000C5
:100F3000000000FFFF00000000FFFF00000000FFB6
:100F40000000000000000000FF00000000FF0000A3
:100F50000000FF00000000FF000000000000FF0094
:100F60000000000000FF000000000000FF00000083
:100F70000000000000000000000000000000000071
:100F8000FFFFFFFFFF000000000000000000000066
:100F90000000FFFFFFFFFF00000000000000000056
:100FA0000000000000FF000000000000FF00000043
:100FB000000000FF000000000000FF00000000FF34
:100FC00000000000FF00000000FF00000000000023
:100FD0000000000000FFFFFF0000FF000000FF0016
:100FE00000000000FF000000FFFF00000000FF0005
:100FF00000000000000000000000FF0000000000F2
:101000000000000000FFFFFF0000FF000000FF00E5
:10101000FF00FFFFFF00FF00FF00FF00FF00FFFFDA
:10102000FF00FF000000000000FFFFFF00000000C5
:101030000000000000FFFFFF0000FF000000FF00B5
:10104000FF000000FF00FF000000FF00FFFFFFFFA8
:10105000FF00FF000000FF00FF000000FF00000095
:1010600000000000FFFFFFFF0000FF000000FF0086
:10107000FF000000FF00FFFFFFFF0000FF00000077
:10108000FF00FF000000FF00FFFFFFFF0000000067
:101090000000000000FFFFFF0000FF000000FF0055
:1010A000FF0000000000FF0000000000FF00000043
:1010B0000000FF000000FF0000FFFFFF0000000035
:1010C00000000000FFFFFFFF0000FF000000FF0026
:1010D000FF000000FF00FF000000FF00FF00000015
:1010E000FF00FF000000FF00FFFFFFFF0000000007
:1010F00000000000FFFFFFFFFF00FF0000000000F6
:10110000FF0000000000FFFFFFFF0000FF000000E5
:101110000000FF0000000000FFFFFFFFFF000000D5
:1011200000000000FFFFFFFFFF00FF0000000000C5
:10113000FF0000000000FFFFFFFF0000FF000000B5
:101140000000FF0000000000FF00000000000000A1
:101150000000000000FFFFFF0000FF000000FF0094
:10116000FF0000000000FF00FFFFFF00FF00000085
:10117000FF00FF000000FF0000FFFFFFFF00000076
:1011800000000000FF000000FF00FF000000FF0063
:10119000FF000000FF00FFFFFFFFFF00FF00000057
:1011A000FF00FF000000FF00FF000000FF00000044
:1011B0000000000000FFFFFF00000000FF00000033
:1011C0000000FF0000000000FF0000000000FF0022
:1011D00000000000FF00000000FFFFFF0000000013
:1011E0000000000000000000FF0000000000FF0001
:1011F00000000000FF0000000000FF00FF000000F2
:10120000FF00FF000000FF0000FFFFFF00000000E4
:1012100000000000FF000000FF00FF0000FF0000D2
:10122000FF00FF000000FFFF00000000FF00FF00C4
:101230000000FF0000FF0000FF000000FF000000B2
:1012400000000000FF0000000000FF0000000000A0
:10125000FF0000000000FF0000000000FF00000091
:101260000000FF0000000000FFFFFFFFFF00000084
:1012700000000000FF000000FF00FFFF00FFFF0074
:10128000FF00FF00FF00FF000000FF00FF00000064
:10129000FF00FF000000FF00FF000000FF00000053
:1012A00000000000FF000000FF00FFFF0000FF0043
:1012B000FF00FF00FF00FF0000FFFF00FF00000035
:1012C000FF00FF000000FF00FF000000FF00000023
:1012D0000000000000FFFFFF0000FF000000FF0013
:1012E000FF000000FF00FF000000FF00FF00000003
:1012F000FF00FF000000FF0000FFFFFF00000000F4
:1013000000000000FFFFFFFF0000FF000000FF00E3
:10131000FF000000FF00FFFFFFFF0000FF000000D4
:101320000000FF0000000000FF00000000000000BF
:101330000000000000FFFFFF0000FF000000FF00B2
:10134000FF000000FF00FF000000FF00FF00FF00A3
:10135000FF00FF0000FF000000FFFF00FF00000093
:1013600000000000FFFFFFFF0000FF000000FF0083
:10137000FF000000FF00FFFFFFFF0000FF0000FF75
:101380000000FF000000FF00FF000000FF00000061
:101390000000000000FFFFFF0000FF000000FF0052
:1013A000FF000000000000FFFFFF00000000000041
:1013B000FF00FF000000FF0000FFFFFF0000000033
:1013C00000000000FFFFFFFFFF000000FF00000023
:1013D0000000FF0000000000FF0000000000FF0010
:1013E00000000000FF0000000000FF0000000000FF
:1013F00000000000FF000000FF00FF000000FF00F1
:10140000FF000000FF00FF000000FF00FF000000E1
:10141000FF00FF000000FF0000FFFFFF00000000D2
:1014200000000000FF000000FF00FF000000FF00C0
:10143000FF000000FF00FF000000FF00FF000000B1
:10144000FF0000FF00FF00000000FF0000000000A0
:1014500000000000FF000000FF00FF000000FF0090
:10146000FF00FF00FF00FF00FF00FF00FF00FF0084
:10147000FF00FF00FF00FF0000FF00FF0000000072
:1014800000000000FF000000FF00FF000000FF0060
:1014900000FF00FF00000000FF00000000FF00FF51
:1014A0000000FF000000FF00FF000000FF00000040
:1014B00000000000FF000000FF00FF000000FF0030
:1014C000FF000000FF0000FF00FF00000000FF0021
:1014D00000000000FF0000000000FF00000000000E
:1014E00000000000FFFFFFFF0000000000FF000001
:1014F0000000FF00000000FF00000000FF000000EF
:101500000000FF0000000000FFFFFFFF00000000E0
:10151000000000000000FFFF000000FF00000000CE
:1015200000FF00000000FFFF0000000000FF0000BF
:10153000000000FF000000000000FFFF00000000AE
:10154000000000000000FFFF000000FF0000FF009F
:10155000FF00FFFF00FFFF00FF0000FFFF00FFFF95
:1015600000FF00FF0000FF000000FFFF0000000080
:101570000000000000FFFF000000000000FF00006E
:10158000000000FF0000000000FFFF00000000FF5F
:101590000000000000FF000000FFFF00000000004E
:1015A0000000000028000E00000001000200020000
:1015B000020002000200020002000200020002001B
:1015C000020002000200020002000200020002000B
:1015D00002000200020002000200020002000200FB
:1015E00002000200020002000200020002000200EB
:1015F00002000200030004000500060006000700C8
:101600000800080009000A000A000B000A000A008E
:101610000B000A000A000B000A000A000B000A0077
:101620000A000B000A000A000B000A000A000B0067
:101630000A000A000B000A000A000C00080008005B
:101640000D00060006000E000500060006000F0053
:1016500010001000110012001200130012001200FE
:1016600013001200120013001200120013001200E7
:1016700012001300120012001300120012001300D7
:1016800012001200130012001200140010001000CB
:101690001500060006000E000500060006000F00FB
:1016A00010001000110012001200130012001200AE
:1016B0001300120012001300120012001300120097
:1016C0001200130012001200130012001200130087
:1016D000120012001300120012001400100010007B
:1016E0001500060006000E000500160017000F008A
:1016F00010001000180019001A001B0019001A0031
:101700001B0019001A001B0019001A001B00190009
:101710001A001B0019001A001B0019001A001B00F8
:1017200019001A001B0019001A001C0010001000FC
:1017300015001D001E000E00050006001F00200001
:1017400010001000210022002300240022002300AA
:101750002400220023002400220023002400220071
:101760002300240022002300240022002300240060
:101770002200230024002200230025001000100076
:101780002600270006000E000500060028000F00B6
:1017900010001000110012001200130012001200BD
:1017A00013001200120013001200120013001200A6
:1017B0001200130012001200130012001200130096
:1017C000120012001300120012001400100010008A
:1017D0001500280006000E000500060029002A005A
:1017E00010001000180019001A001B0019001A0040
:1017F0001B0019001A001B0019001A001B00190019
:101800001A001B0019001A001B0019001A001B0007
:1018100019001A001B0019001A001C00100010000B
:101820002B002C0006000E0005002D002E000F00DE
:1018300010001000210022002300240022002300B9
:101840002400220023002400220023002400220080
:10185000230024002200230024002200230024006F
:101860002200230024002200230025001000100085
:1018700015002F0030000E000500060006000F00C6
:1018800010001000110012001200130012001200CC
:1018900013001200120013001200120013001200B5
:1018A00012001300120012001300120012001300A5
:1018B0001200120013001200120014001000100099
:1018C0001500060006000E000500060006000F00C9
:1018D000100010001100120012001300120012007C
:1018E0001300120012001300120012001300120065
:1018F0001200130012001200130012001200130055
:101900001200120013001200120014001000100048
:101910001500060006000E00050006000600310056
:10192000320032003300340034003500340034001B
:101930003500340034003500340034003500340004
:1019400034003500340034003500340034003500F4
:1019500034003400350034003400360032003200E8
:101960003700060006000E00380039003A003A0041
:101970003A003A003A003A003A003A003A003A0097
:101980003A003A003A003A003A003A003A003A0087
:101990003A003A003A003A003A003A003A003A0077
:1019A0003A003A003A003A003A003A003A003A0067
:1019B0003A003A003B003C001200120012001200F4
:1019C0001200120012001200120012001200120087
:1019D0001200120012001200120012001200120077
:1019E0001200120012001200120012001200120067
:1019F0001200120012001200120012001200120057
:101A0000120012001200120022000900120012003F
:101A10001200120012001200120012001200120036
:101A20001200120012001200120012001200120026
:101A3000120012001200120012003D003E003F0092
:101A40001200120012001200120012001200120006
:101A50001200120012001200400041004200430038
:101A600044004500460047004300480049004A0042
:101A70004B004C004D0012004E004F005000510032
:101A8000520053005400550056001200120012007C
:101A9000120012001200120012001200570058002B
:101AA00059005A005B005C005D005E005F00600052
:101AB0005900610062006300640012006500660066
:101AC0006700680069006A006B006C006D0012001E
:101AD0001200120012001200120012001200120076
:101AE0006E006F007000710072007300740075006A
:101AF00076007700780079007A007B007C00120085
:101B000012007D007E007F00800081008200830043
:101B10001200120012001200120012001200120035
:101B2000120012008400850086008700880089006A
:101B30008A008B0087008C008D008E008F00900043
:101B400091009200930094001200120095009600FC
:101B500097009800120099009A00120012001200DB
:101B600012001200120012009B009C009D009E00BB
:101B70009F00A000A100A200A300A400A500A60051
:101B8000A700A800A900AA00AB00AC00AD00AE0001
:101B9000AF00B000B100B2001200B300B4001200F8
:101BA000120012001200120012001200B500B6005E
:101BB000B700B800B9001200BA00BB00B200BC0008
:101BC0001200BD00BE00BF00B400C000C100C200D2
:101BD000C300C400C500C600C700B2001200B300B5
:101BE000B4001200120012001200120012001200C3
:101BF000C800C9001200CA00CB00CC00CD00CE0046
:101C0000CF00D000D100D200D300BF00B400C0008C
:101C1000D400D500D600D700D800D900DA00DB0008
:101C2000DC00DD00DE00DC00DF001200120012002C
:101C300012001200E000E10012001200E200E300D6
:101C4000E4001200E500E600E300E7001200E8000F
:101C5000E900E500EA00E300E700E000EB00EC004B
:101C6000E900ED00E300E100E200E300EE00120015
:101C70002D2D2D2D2D2D2D2D2D2D2D2D2D2D2D2D94
:101C80002D2D2D2D2D2D2D2D2D2D2D2D2D2D2D2D84
:101C90002D2D2D2D2D2D2D2D2D182D2D2D2D2D189E
:101CA0002D2D2D2D2D2D2D2D2D2D2D2D2D2D2D2D64
:101CB0002D2D2D2D2D2D2D2D2D2D2D2D2D2D2D1869
:101CC0001818181818181818181818181818181894
:101CD0002D2D2D2D2D2D2D2D2D2D2D2D2D2D2D2D34
:101CE0002D2D2D2D2D2D2D2D2D2D2D2D2D2D18184E
:101CF0001818181818181818181818181818181864
:101D00002D2D2D2D2D2D2D2D2D2D2D2D2D2D2D2D03
:101D10002D2D2D2D2D2D2D2D2D2D2D2D2D2D18181D
:101D20001818182D1818181818181818181818181E
:101D30002D2D2D2D2D2D2D2D2D2D2D2D2D2D2D2DD3
:101D40002D2D2D2D2D2D2D2D2D2D2D2D2D2D2D2DC3
:101D50002D2D2D2D182D2D2D2D2D182D2D2D2D2DDD
:101D60002D2D2D2D18182D2D2D2D18182D2D2D2DF7
:101D700018182D2D2D2D18182D2D2D2D18182D2D11
:101D80002D2D18182D2D2D2D18182D2D2D2D181801
:101D900018181818181818181818181818181818C3
:101DA00018181818181818181818181818181818B3
:101DB00018181818181818181818181818181818A3
:101DC0001818181818181818181818181818181893
:101DD00018181818FFFFFFFF1818FFFFFFFF18184B
:101DE000FFFFFFFF1818FFFFFFD81818FFFFFFD8ED
:101DF0001818181818181818181818181818181863
:101E00001818FFFFFFFFFFFFFFFFFFFFFFFFFFFFB0
:101E1000FFFFFFFFD8D8D8D8D8D8D8D8D8D8D8D8A6
:101E20001818181818181818181818181818181832
:101E30001818FFFFFFFFFFFFFFFFFFFFFFFFFFFF80
:101E4000FFFFFFFFD8D8FFFF0000D8D8FFFF00003A
:101E50001818181818181818181818181818181802
:101E60001818FFFFFFFFFFFFFFFFFFFFFFFFFFFF50
:101E7000FFFFFFFF00000000000000000000000066
:101E800018181818181818181818181818181818D2
:101E90001818FFFFFFFFFFFFFFFFFFFFFFFFFFFF20
:101EA000FFFFFFFF0000FFFF00000000FFFF00003A
:101EB00018181818181818181818181818181818A2
:101EC0001818FFFFFFFFFFFFFFFFFFFFFFFFFFFFF0
:101ED000FFFFFFFF0000FFFFD8D80000FFFFD8D8AA
:101EE0001818181818181818181818181818181872
:101EF0001818FFFFFFFF1818FFFFFFFF1818FFFF5C
:101F0000FFFF1818D8FFFFFF1818D8FFFFFF181899
:101F100018182D2D2D2D18182D2D2D2D18182D2D6F
:101F20002D2D18182D2D2D2D18182D2D2D2D18185F
:101F30002D2D2D2D18182D2D2D2D18182D2D2D2D25
:101F40001818FFFFFFD81818FFFFFFD81818FFFF59
:101F5000FFD81818FFFFFFD81818FFFFFFD8181870
:101F6000FFFFFFD81818FFFFFFD81818FFFFFFD892
:101F7000D8D8D8D8D8D8D8D8D8D8D8D8D8D8D8D8E1
:101F8000D8D8D8D8D8D8D8D8D8D8D8D8D8D8D8D8D1
:101F9000D8D8D8D8D8D8D8D8D8D8D8D8D8D8D8D8C1
:101FA000D8D8FFFF0000D8D8FFFF0000D8D8FFFF27
:101FB0000000D8D8FFFF0000D8D8FFFF0000D8D815
:101FC000FFFF0000D8D8FFFF0000D8D8FFFF0000B7
:101FD0000000000000000000000000000000000001
:101FE00000000000000000000000000000000000F1
:101FF00000000000000000000000000000000000E1
:102000000000FFFF00000000FFFF00000000FFFFD6
:1020100000000000FFFF00000000FFFF00000000C4
:10202000FFFF00000000FFFF00000000FFFF0000B6
:102030000000FFFFD8D80000FFFFD8D80000FFFF46
:10204000D8D80000FFFFD8D80000FFFFD8D8000084
:10205000FFFFD8D80000FFFFD8D80000FFFFD8D876
:10206000D8FFFFFF1818D8FFFFFF1818D8FFFFFF91
:102070001818D8FFFFFF1818D8FFFFFF1818D8FF4F
:10208000FFFF1818D8FFFFFF1818D8FFFFFF181818
:10209000181818181818181818181818181818FFD9
:1020A0001818181818FFFF1818181818FFFF181814
:1020B000181818FF181818181818181818181818B9
:1020C0001818181818181818181818181818181890
:1020D0001818181818181818181818181818FF1899
:1020E00018181818FFFF1818181818FFFF181818D4
:1020F000D8D8FFFF0000D8D8FFFF0000D8D8FFFFD6
:102100000000D8D8FFFF0000D8D8FFFF0000D8D8C3
:10211000FFFF0000D8D8FFFF0000D8D8FFFFFFFF67
:1021200000000000000000000000000000000000AF
:10213000000000000000000000000000000000009F
:1021400000000000000000000000FFFFFF00000092
:10215000000000000000000000000000000000007F
:10216000000000000000000000000000000000006F
:1021700000000000000000000000000000FFFFFF62
:102180000000FFFF00000000FFFF00000000FFFF55
:1021900000000000FFFF00000000FFFF0000000043
:1021A000FFFF00000000FFFF0000FFFFFFFFFFFF39
:1021B0000000FFFFD8D80000FFFFD8D80000FFFFC5
:1021C000D8D80000FFFFD8D80000FFFFD8D8000003
:1021D000FFFFD8D80000FFFFD8D8FFFFFFFFD8D8F7
:1021E000181818181818181818181818181818186F
:1021F000181818181818181818181818181818185F
:10220000181818181818181818FF18181818FFFF99
:10221000181818181818181818181818181818183E
:1022200018181818FF18181818FFFF181818FFFFAB
:1022300018181818FF181818181818181818181837
:102240001818FFFF18181818FFFFFF181818FFFFBD
:10225000FFFF1818FFFF18FF1818FFFF18181818AD
:10226000FFFF18181818FFFF18181818FFFF181884
:102270001818FFFFFFD81818FFFFFFD81818FFFF26
:10228000FFD8FF18FFFFFFD8FFFFFFFFFFD818FFA1
:10229000FFFFFFD81818FFFFFFD81818FFFFFFD85F
:1022A000D8D8FFFFFFFFD8D8FFFF0000D8D8FFFF26
:1022B0000000D8D8FFFF0000D8D8FFFF0000D8D812
:1022C000FFFF0000D8D8FFFF0000D8D8FFFF0000B4
:1022D000FFFFFF0000000000000000000000000001
:1022E00000000000000000000000000000000000EE
:1022F00000000000000000000000000000000000DE
:10230000000000FFFFFF00000000000000000000D0
:1023100000000000000000000000000000000000BD
:1023200000000000000000000000000000000000AD
:10233000FFFFFFFFFFFF0000FFFF00000000FFFFA7
:1023400000000000FFFF00000000FFFF0000000091
:10235000FFFF00000000FFFF00000000FFFF000083
:10236000FFFFFFFFD8D80000FFFFD8D80000FFFF15
:10237000D8D80000FFFFD8D80000FFFFD8D8000051
:10238000FFFFD8D80000FFFFD8D80000FFFFD8D843
:10239000D8FFFFFF1818D8FFFFFF1818D8FFFFFF5E
:1023A0001818D8FFFFFF1818D8FFFFFF18FFD8FF35
:1023B000FFFFFFFFD8FFFFFFFF18D8FFFFFF181830
:1023C000181818FFFF181818FFFF181818FFFFFF3C
:1023D0001818FFFFFFFF1818FF18FFFF181818182C
:1023E000FFFF18181818FFFF18181818FFFF181803
:1023F0001818FFFF18181818FFFF18181818FFFFF3
:1024000018181818FFFF18181818FFFF18181818B0
:10241000FFFF18181818FFFF18181818FFFF1818D2
:102420001818FFFF18181818FFFF18181818FFFFC2
:1024300018181818FFFF18FF1818FFFFFFFF1818CB
:10244000FFFFFF181818FFFF181818FFFF181818BB
:102450001818FFFFFFD818FFFFFFFFD8FFFFFFFF8F
:10246000FFD8FF18FFFFFFD81818FFFFFFD8181874
:10247000FFFFFFD81818FFFFFFD81818FFFFFFD87D
:10248000D8FFFFFF1818D8FFFFFF1818D8FFFFFF6D
:10249000FF18D8FFFFFFFFFFD8FFFFFF18FFD8FF8F
:1024A000FFFF1818D8FFFFFF1818D8FFFFFF1818F4
:1024B0001818FFFF18181818FFFF18181818FFFF32
:1024C00018181818FFFF1818FF18FFFF1818FFFF3B
:1024D000FFFF181818FFFFFF18181818FFFF18182B
:1024E0001818181818181818181818FF1818181885
:1024F000FFFF181818FFFF18181818FF18181818D9
:10250000181818181818181818181818181818184B
:10251000FFFF18181818FF18181818181818181886
:10252000181818181818181818181818181818182B
:10253000181818181818181818181818181818181B
:10254000181818FFFF1818181818FFFF181818186F
:1025500018FF181818181818181818181818181814
:1025600018181818181818181818181818181818EB
:10257000181818181818181818181818FF181818F4
:102580001818FFFF1818181818FFFF18181818182F
:10259000FF181818181818181818181818181818D4
:1025A0001818FFFFFFD81818FFFFFFD81818FFFFF3
:1025B000FFFF1818FFFFFFFF1818FFFFFFFF181895
:1025C000181818181818181818181818181818188B
:1025D000D8D8D8D8D8D8D8D8D8D8D8D8FFFFFFFFDF
:1025E000FFFFFFFFFFFFFFFFFFFFFFFFFFFF1818C9
:1025F000181818181818181818181818181818185B
:10260000D8D8FFFF0000D8D8FFFF0000FFFFFFFF72
:10261000FFFFFFFFFFFFFFFFFFFFFFFFFFFF181898
:10262000181818181818181818181818181818182A
:10263000000000000000000000000000FFFFFFFF9E
:10264000FFFFFFFFFFFFFFFFFFFFFFFFFFFF181868
:1026500018181818181818181818181818181818FA
:102660000000FFFF00000000FFFF0000FFFFFFFF72
:10267000FFFFFFFFFFFFFFFFFFFFFFFFFFFF181838
:1026800018181818181818181818181818181818CA
:102690000000FFFFD8D80000FFFFD8D8FFFFFFFFE2
:1026A000FFFFFFFFFFFFFFFFFFFFFFFFFFFF181808
:1026B000181818181818181818181818181818189A
:1026C000D8FFFFFF1818D8FFFFFF1818FFFFFFFF04
:1026D0001818FFFFFFFF1818FFFFFFFF1818181842
:1026E000181818181818181818181818181818186A
:1026F0002D2D2D2D2D182D2D2D2D2D182D2D2D2D34
:102700002D2D2D2D2D2D2D2D2D2D2D2D2D2D2D2DF9
:102710002D2D2D2D2D2D2D2D2D2D2D2D2D2D2D2DE9
:102720001818181818181818181818182D18181814
:1027300018182D2D2D2D2D2D2D2D2D2D2D2D2D2DF3
:102740002D2D2D2D2D2D2D2D2D2D2D2D2D2D2D2DB9
:1027500018181818181818181818181818181818F9
:1027600018182D2D2D2D2D2D2D2D2D2D2D2D2D2DC3
:102770002D2D2D2D2D2D2D2D2D2D2D2D2D2D2D2D89
:1027800018181818181818181818181818181818C9
:10279000182D2D2D2D2D2D2D2D2D2D2D2D2D2D2D7E
:1027A0002D2D2D2D2D2D2D2D2D2D2D2D2D2D2D2D59
:1027B000182D2D2D2D2D182D2D2D2D2D2D2D2D2D73
:1027C0002D2D2D2D2D2D2D2D2D2D2D2D2D2D2D2D39
:1027D0002D2D2D2D2D2D2D2D2D2D2D2D2D2D2D2D29
:1027E00000000000000000000000000000000000E9
:1027F00000000000000000000000000000000000D9
:1028000000000000000000000000000000000C0CB0
:1028100000000000000000000000000000000000B8
:1028200000000000000000000000000000000000A8
:10283000000000000000000000000C0C0C0C0C0C50
:102840000000000000000000000000000000000088
:102850000000000000000000000000000000000078
:10286000000000000000000000000C0C0C00000044
:102870000000000000000000000000000000000058
:1028800000000000000000FF00000000FFFF00004B
:102890000000FFFF00000000FFFF00000000FFFF3E
:1028A0000000000000000000000000000000000028
:1028B0000000000000000000FF0000000000FF001A
:1028C00000000000FF0000000000FF00000000000A
:1028D00000000000000000000000000000000000F8
:1028E000000000FF00000000FFFFFF0000FFFFFFEF
:1028F000FF000000FFFFFF000000FFFFFF000000DF
:1029000000000000000000000000000000000000C7
:102910000000FFFFFFFFFFFFFFFFFFFFFFFFFFFFC5
:10292000FFFFFFFF000000000000000000000000AB
:102930000000000000000000000000000000000097
:102940000000FFFFFFFFFF00FFFFFFFFFFFFFFFF94
:10295000FFFFFFFF00FFFFFFFFFFFFFFFFFFFFFF86
:102960000000000000000000000000000000000067
:10297000000000000000FFFF000000FFFFFF00005C
:1029800000FFFFFF000000FFFFFF000000FFFFFF50
:102990000000000000000000000000000000000037
:1029A0000000FFFFFFFFFFFFFFFFFFFFFFFFFFFF35
:1029B000FFFFFFFFFF0000000000FF00000000001D
:1029C0000000000000000000000000000000000007
:1029D00000000000000000FFFF000000FFFF0000FB
:1029E0000000FFFF00000000FFFF00000000FFFFED
:1029F00000000000000000000000000000000000D7
:102A00000000000000000000FF0000000000FFFFC9
:102A100000000000FFFFFF000000FFFFFF000000BC
:102A200000000000000000000000000000000000A6
:102A3000000000FFFFFFFFFFFFFFFFFFFFFFFFFFA3
:102A4000FFFFFFFFFFFFFFFFFFFFFFFFFF00000093
:102A50000000000000000000000000000000000076
:102A60000000FFFFFFFFFF00FFFFFFFFFFFFFFFF73
:102A7000FFFFFFFFFFFFFFFFFFFF000000FFFFFF63
:102A80000000000000000000000000000000000046
:102A90000000000000FFFFFF000000FFFFFF00003C
:102AA00000FFFFFF000000FFFFFF00000000FFFF2E
:102AB0000000000000000000000000000000000016
:102AC00000000000000000000000000000FF000007
:102AD000000000FF0000000000FFFF000000FFFFFB
:102AE00000000000000000000000000000000000E6
:102AF0000000FFFFFF000000FFFFFF000000FFFFDE
:102B0000FF000000FFFFFF000000FFFF00000000CB
:102B100000000000000000000000000000000000B5
:102B200000000000000000000000000000000000A5
:102B30000000000C000000000C0C000000000C0C59
:102B40000000000000000000000000000000000085
:102B50000CFF00000C0CFFFF000C0CFFFFFF0C0C27
:102B60000CFFFFFF0C0C0CFFFFFF0C0C0CFFFFFF1A
:102B7000000000000C0C000C0C0C0C0CFF0C0C0CDE
:102B80000C0C0C0C0C0C0C0C0C0C0C0C0C0C0C0C85
:102B90000C0C0C0C0C0C0C0CFF0C0C0C0C0CFF0C8F
:102BA0000C0C0C0C0C0C0C0C0C0C0C0C0C0C0C0C65
:102BB0000C0C0C0C0C0C0C0C0C0C0C0C0C0C0C0C55
:102BC0000C0CFF0C0CFF0C0CFF0C0CFFFFFFFFFFAD
:102BD0000C0C0C0C0C0C0C0C0C0C0C0C0C0C0C0C35
:102BE0000C0C0C0C0C0C0C0C0C0C0C0C0C0C0CFF32
:102BF0000C0CFF0C0CFF0C0CFF0CFFFFFFFFFFFF8A
:102C00000C0C0C0C0C0C0C0C0C0C0C0C0C0C0C0C04
:102C10000C0C0C0C0C0C0C0C0C0C0C0C0C0C0CFF01
:102C20000C0C0C0C0CFF0C0CFF0CFFFFFFFFFF0C3F
:102C30000C0C0C0000000C0C0C0C0C0C0C0C0C0CF8
:102C40000C0C0C0C0C0C0C0C0C0C0C0C0C0C0C0CC4
:102C50000C0C0C0C0CFF0C0C0C0C0CFF0C0C0C0CCE
:102C6000000000000000000000000000FFFF0C005A
:102C700000000CFFFF0C0C000CFFFFFF0C0C0CFF06
:102C8000FFFF0C0C0CFFFFFF0C0C0CFFFFFF0C0CEC
:102C90000000000000000000000000000000000034
:102CA00000000000000000000000000000000C0C0C
:102CB000000000000C0C0C0000000C0C0C000000CC
:102CC00000000000FFFF00000000FFFF0000000008
:102CD000FFFF00000000FFFF000000FFFFFF0000FB
:102CE00000FFFFFF000000FFFFFF000000FFFFFFED
:102CF000FF0000000000FF0000000000FF000000D7
:102D00000000FF0000000000FF0000000000FF00C6
:102D100000000000FF0000000000FF0000000000B5
:102D2000FFFFFF000000FFFFFF000000FFFFFF00AC
:102D30000000FFFFFF000000FFFFFF000000FFFF9B
:102D4000FF000000FFFFFF000000FFFFFF0000008A
:102D50000000000000000000000000000000000073
:102D600000FF0000000000FF00000000FFFF000067
:102D70000000FFFF000000FFFFFF000000FFFFFF5B
:102D8000FFFFFFFFFF00FFFFFFFF0000FFFFFFFF50
:102D90000000FFFFFF000000FFFFFF000000FFFF3B
:102DA00000000000FFFF00000000FF000000000026
:102DB000000000FFFFFF000000FFFFFF000000FF1A
:102DC000FFFF000000FFFFFF000000FFFFFF00000B
:102DD000FFFFFFFF0000FFFFFFFF0000FFFFFFFFFF
:102DE000FF0000000000FF0000000000FF000000E6
:102DF0000000FF0000000000FFFFFFFFFF00FFFFDB
:102E0000FFFFFFFFFFFFFFFFFF00FF0000000000CC
:102E100000000000FFFF00000000FFFF00000000B6
:102E2000FFFF00000000FFFF00000000FFFF0000A8
:102E300000FFFFFF000000FFFFFF000000FFFFFF9B
:102E40000000000000000000000000000000000082
:102E50000000000000000000000000000000000072
:102E600000000000FFFFFFFFFFFFFFFFFFFFFFFF6E
:102E7000FFFFFF000000FFFFFF000000FFFFFF005B
:102E80000000FFFFFF000000FFFFFF000000FFFF4A
:102E900000000000FFFF000000FFFFFFFF0000FF39
:102EA000000000FFFFFF000000FFFFFF000000FF29
:102EB000FFFF000000FFFFFF000000FFFFFF00001A
:102EC00000FFFFFF000000FFFFFF000000FFFFFF0B
:102ED00000000000FFFF00000000FFFF00000000F6
:102EE000FFFF00000000FFFF0000000000FF0000E7
:102EF000000000FF0000000000FF000000FFFFFFD7
:102F0000FF000000FFFFFF000000FFFFFF000000C8
:102F1000FFFFFF000000FFFFFFFFFFFFFFFFFFFFBE
:102F2000FFFFFFFFFFFFFFFFFFFFFFFFFFFFFFFFB1
:102F3000FFFF00000000FF0000000000FF00000095
:102F40000000FF0000000000000000000000000082
:102F50000000000000000000000000000000000071
:102F60000000000C0C0C0000000C0C0C0000000B0E
:102F70000B0B0000000C0C0C000000000C0C0000FF
:102F800000000C0C00000000000C0000000000001D
:102F90000C0C0CFFFFFF0C0B0BFFFFFF0B0C0CFFCF
:102FA000FFFF0C0C0CFFFFFF0C0C0CFFFFFF0C0CC9
:102FB0000CFFFFFF0C0C0CFFFFFF000C0CFFFFFFD2
:102FC0000C0C0BFFFFFF0B0B0CFFFFFF0C0C0C0C92
:102FD000FF0C0C0C0C0CFF0C0C0C0C0C0C0C0C0C4B
:102FE0000C0C0C0C0C0C0C0C0C0C0C0C0C0C0C0C21
:102FF000FFFFFFFFFFFFFFFF0C0CFF0C0CFF0C0C93
:10300000FF0C0CFF0C0C0C0C0C0C0C0C0C0C0C0C1A
:103010000C0C0C0C0C0C0C0C0C0C0C0C0C0C0C0CF0
:10302000FFFFFFFFFFFF0CFF0C0CFF0C0CFF0C0C55
:10303000FF0C0C0C0C0C0C0C0C0C0C0C0C0C0C0CDD
:103040000C0C0C0C0C0C0C0C0C0C0C0C0C0C0C0CC0
:10305000FFFFFFFFFFFF0CFF0C0CFFFF0CFF0C0C32
:10306000FF0C0C0C0C0CFF0C0C0C0C0C0C0C0C0CBA
:103070000C0C0C0C0C0C0C0C0C0C0C0C0C0C0C0C90
:10308000FFFFFF0B0C0CFFFFFF0C0B0B0CFF0C0CDE
:103090000C0C0CFF0C0C0C0C0C0C0C0C0C0C0C0C7D
:1030A0000C0C0C0C0C0C0C0C0C0C0C0C0C0C0C0C60
:1030B0000CFFFFFF0C0C0BFFFFFF0B0C0CFFFFFFC7
:1030C0000C0B0CFFFFFF0C0C0CFFFFFF0C0C0CFF9C
:1030D000FFFF0C0C0CFFFFFF0C0C0CFFFFFF0C0C98
:1030E0000C0C0C0C00000C0C0C0C00000B0B0B0B54
:1030F00000000C0C0C0C00000C0C0C0000000C0C64
:103100000C0000000C0C000000000000000000009B
:103110000000FFFFFFFF0000FFFFFFFF0000FFFFB9
:10312000FFFF0000FFFFFFFF0000FFFFFFFF0000A9
:10313000FFFFFFFF000000FFFFFF00000000FFFF98
:10314000FF0000000000FF0000000000FF00000082
:103150000000FF0000000000FF0000000000FFFF73
:10316000000000FFFFFFFFFFFFFFFFFFFFFFFFFF6C
:10317000FFFFFF000000FFFFFF000000FFFFFF0058
:1031800000FFFFFFFF0000FFFFFFFF00FFFFFFFF4B
:10319000FF00FFFFFFFFFF00FFFFFFFFFF00FFFF3C
:1031A00000FFFFFFFFFFFFFFFFFFFFFFFFFFFFFF2E
:1031B000FF00FFFFFFFF0000FFFFFFFF0000FFFF1A
:1031C000FFFF0000FFFFFFFFFFFFFFFFFFFFFFFF0D
:1031D000FF000000000000000000000000000000F0
:1031E00000000000000000000000000000000000DF
:1031F00000000000FFFFFFFFFF00FFFFFFFFFFFFDA
:103200000000FFFFFFFF00FFFFFFFFFF00FFFFFFCA
:10321000FFFF00FFFFFFFFFF00FFFFFFFFFF00FFBB
:10322000FFFFFFFF00FFFFFFFFFF00FFFFFFFFFFAC
:10323000FF0000000000FF0000000000FF00000091
:103240000000FF0000000000FF0000000000FF0081
:1032500000000000FFFFFFFFFFFFFFFFFFFFFFFF7A
:10326000000000FFFFFF000000FFFFFF0000FFFF66
:10327000FFFF0000FFFFFFFF0000FFFFFFFF000058
:10328000FFFFFFFF0000FFFFFFFFFF00FFFFFFFF4B
:10329000FFFFFFFFFFFF0000000000000000000034
:1032A000000000000000000000000000000000001E
:1032B00000000000FFFFFFFFFFFFFFFFFFFFFFFF1A
:1032C000FFFFFF0000FFFFFFFF00FFFFFFFFFF000A
:1032D000FFFFFFFFFF00FFFFFFFFFF00FFFFFFFFFC
:1032E000FF00FFFFFFFFFF00FFFFFFFF0000FFFFEA
:1032F000FFFFFF000000FFFFFF000000FFFFFF00D7
:103300000000FFFFFF000000FFFFFF000000FFFFC5
:10331000FF000000FFFFFFFFFFFFFFFFFFFFFFFFBA
:10332000000000FFFFFF000000FFFFFF000000FFA4
:10333000FFFF000000FFFFFF000000FFFFFF000095
:1033400000FFFFFFFFFFFFFFFFFFFFFFFFFFFFFF8C
:10335000000000FFFFFF0000FFFFFFFF0000FFFF76
:10336000FFFF0000FFFFFFFF00FFFFFFFFFF00FF69
:10337000FFFFFFFF00FFFFFFFFFF00FFFFFFFFFF5B
:10338000FFFFFFFFFFFFFF000000FFFFFF00000047
:10339000FFFFFF000000FFFFFF000000FFFFFF0036
:1033A000000000FF0000000000FF0000000000001F
:1033B000FF0000000000FF0000000000FF00000010
:1033C0000000FFFF00000000FFFF00000000FFFF03
:1033D000FF000000FFFFFF000000FFFFFF000000F4
:1033E00000000C0CFFFF000000000CFF00000000BC
:1033F00000000000000000000000000000000000CD
:1034000000000000000000000000000000000000BC
:103410000C0C0C0C0C0CFF0C0C0C0C0CFF0C0C0C06
:103420000C0C000000000C0C00000000000000006C
:10343000000000000000000000000000000000008C
:103440000C0C0C0C0C0C0C0C0C0C0C0C0C0C0C0CBC
:103450000C0C0C0C0C0C0C0C000000000C0C0000F4
:10346000000000000000000000000000000000005C
:103470000C0C0C0C0C0C0C0C0C0C0C0C0C0C0C0C8C
:103480000C0C0C0C0C0C0C0C0C0C0C0C0C0C000094
:10349000000000000000000000000000000000002C
:1034A0000C0C0C0C0C0C0C0C0C0C0C0C0C0C0C0C5C
:1034B0000C0C0C0C0C0C0C0C0C0C0C000000000088
:1034C00000000000000000000000000000000000FC
:1034D0000C0C0C0C0C0C0C0C0C0C0C0C0C0C0C0C2C
:1034E0000C0C0C0C0C0000000000000000000000A0
:1034F00000000000000000000000000000000000CC
:103500000CFFFF0C0C00FFFF0C000000FF00000090
:1035100000000000000000000000000000000000AB
:10352000000000000000000000000000000000009B
:103530000000000000FF000000000000000000008C
:10354000000000000000000000000000000000007B
:103550000000000000000000000000000000000764
:10356000FFFFFFFFFFFF0000000000000000000061
:10357000000000000000000000000000000000004B
:103580000000000000000000000007070707070711
:10359000FFFF0000FFFF000000000000000000002F
:1035A000000000000000000000000000000000001B
:1035B00000000000000000000000070707070700E8
:1035C000FFFFFFFFFFFF0000000000000000000001
:1035D00000000000000000000000000000000000EB
:1035E00000000000000000000000000000000000DB
:1035F000FFFFFFFFFF0000000000000000000000D0
:1036000000000000000000000000000000000000BA
:103610000000000000000000070700070707070779
:103620000000FFFFFFFF000000000000000000009E
:10363000000000000000000000000000000000008A
:10364000000000000707070707000707070707072D
:10365000FFFFFFFFFFFF0000000000000000000070
:10366000000000000000000000000000000000005A
:10367000000000000000000000000707000000003C
:103680000000FFFFFFFF000000000000000000003E
:10369000000000000000000000000000000000002A
:1036A000000000000000000000000000000000001A
:1036B000FF00000000FF000000000000000000000C
:1036C00000000000000000000000000000000000FA
:1036D00000000000000000070707070707070707AB
:1036E000FFFFFFFFFFFF00000000000000000000E0
:1036F00000000000000000000000000000000000CA
:103700000000000007070707000007070707070773
:10371000FFFFFFFFFF0000000000000000000000AE
:103720000000000000000000000000000000000099
:103730000000000000000000000007000000000082
:1037400000FFFFFFFF00000000000000000000007D
:103750000000000000000000000000000000000069
:10376000000000000000000000000000000007074B
:103770000000000000000000000000000000000049
:103780000000000000000000000000000000000039
:1037900000000000000000000000070707070707FF
:1037A00000FFFFFF0000000000000000000000001C
:1037B0000000000000000000000000000000000009
:1037C00000000000000000000000070707070707CF
:1037D00000000000000000000000000000000000E9
:1037E00000000000000000000000000000000000D9
:1037F00000000000000000000000070707070000AD
:1038000000000000000000000000000000000000B8
:1038100000000000000000000000000000000000A8
:10382000000000000000000000070000000707077C
:103830000000000000000000000000000000000088
:103840000000000000000000000000000000000078
:103850000000000007070707000007070707070722
:103860000000000000000000000000000000000058
:103870000000000000000000000000000000000048
:10388000000000000000000000000000070707071C
:103890000000000000000000000000000000000028
:1038A0000000000000000000000000000000000018
:1038B00000000000000000000000070707000000F3
:1038C00000000000000000000000000000000000F8
:1038D00000000000000000000000000000000000E8
:1038E00000000000000000000007000000000007CA
:1038F00000000000000000000000000000000000C8
:1039000000000000000000000000000000000000B7
:103910000000000007070007070707070007070761
:103920000000000000000000000000000000000097
:103930000000000000000000000000000000000087
:10394000000000000000000707070000000707074D
:103950000000000000000000000000000000000067
:103960000000000000000000000000000000000057
:10397000000000000007070700000007070700001D
:103980000000000007070000000707070000070706
:1039900007070007070707070007070707000007D3
:1039A00007070007000707070007000707070007CA
:1039B00007070707070707070707070707000000AC
:1039C000000000070707070707070707070707079C
:1039D00007070707070700000000070700000000AF
:1039E0000707070707000707070707000000000091
:1039F0000000070707070700070707070700070773
:103A000007070700000000000000000000000000A1
:103A1000000000000007000000000707000000078A
:103A20000707000007070707000707070707000742
:103A3000070707000707070700070707070700072B
:103A40000707070707070707070700000707000022
:103A50000707070007070707000707070707070704
:103A60000707070707070707000007070700000009
:103A700007070707070700000000000707070707F9
:103A800007000707070707070707070707070000DB
:103A90000707070700000000000700000000000003
:103AA00007070700000007070707070007070707C2
:103AB00007070000070707070707000707070707AB
:103AC000070007070707070007070707070700079B
:103AD00000000000000000000000000000000000E6
:103AE00000000700000000000700000000000707BA
:103AF000000000000707000000000707070000079C
:103B0000000000000007000000070707000007078B
:103B1000070700070707070700070707070007074A
:103B2000070700070707070700070707070007073A
:103B30000707070707070707070700000707000031
:103B40000707000007070707070707070707070713
:103B50000707070707070700000007070000000026
:103B60000707070707070000000007070707070701
:103B700000000707070707070707070707070000F1
:103B8000070707070000000007070000000000000B
:103B900007070700000007070707000007070707D8
:103BA00007000000070707070707000707070707C1
:103BB00000070707070707000707070707070007AA
:103BC00000000000070700000000070700000000D9
:103BD00000000000000007070700000007070700BB
:103BE00000000707070700000000070700000000AB
:103BF0000707070707070707070707070000000071
:103C00000000070707070707070707070707070752
:103C1000070707070000000007070000000007076C
:103C20000707070707070707070707070000000040
:103C30000000000707070707000707070707000737
:103C4000070707070007070700000007070700002E
:103C5000070707070000070707070000000000002C
:103C60000000070707070000070707070007070707
:103C70000707000700000000000700000000000721
:103C800000000707070700070707070007070707E0
:103C900000070707070007070707070007070707C9
:103CA00007000707070707000707070707000707B9
:103CB00007070707070700000000070707070707B0
:103CC00000070707070707000707070707000000A7
:103CD0000707070000000707000707070707000797
:103CE00007000000000007070000000007070700AA
:103CF000000007070700000007070700000007078C
:103D00000700000007070700000007070700000082
:103D100000000000000000000000000000000000A3
:103D2000000700000000000700000000000700007E
:103D30000000070700000000070700000000070759
:103D4000000707070707070707070707070707070A
:103D5000000007070700070707070007070707070F
:103D600000070707070700070707070007070700FF
:103D700007070707000007070707070000070707EF
:103D800007000700070707070707000707070707D8
:103D900000070707070700070707070707000707C8
:103DA0000000000000070000000000070000000005
:103DB00000070000000000070000000000070000EE
:103DC00000000007000000000007070000000007D7
:103DD0000707000707070707000707070707000788
:103DE0000707070700070707070700070707070771
:103DF0000007070707070007070707070007070768
:103E00000000000707070000000707070000000781
:103E1000070700000007070700000007070700006A
:103E20000007070700000007070700000007070753
:103E30000007070700000007070700000007070743
:103E40000000000707070000000707070000000741
:103E5000070700000007070700000007070700002A
:103E60000007070700070007070700070007070705
:103E70000007000707070007000707070000000703
:103E800007070007000707070007000707070007E5
:103E900007070000000007070707070707070707CE
:103EA00007070707070707070000000000000707CC
:103EB0000707070707070707070707070707070792
:103EC00000000000000007070700000707070700C1
:103ED00000070707070000070000000000070707AA
:103EE000070000070707070000070707070000078C
:103EF0000707070007070707000707070707000767
:103F0000070707070007070707070007070707074F
:103F10000007070707070007070707070007070746
:103F20000707000000000700000000000700000075
:103F3000000000000000000000000000000007007A
:103F40000000000007000000000007000000000063
:103F50000007070700070000070707000000070722
:103F60000700000007070700000007070700000020
:103F70000707070000000707070000000707070002
:103F800007070700000707070700000707070700E4
:103F900000070707070000070707070000070707D4
:103FA00007000007070707000007070707000007CB
:103FB00007000000000007000000000000000000F3
:103FC00000000000000000000000000000000000F1
:103FD00000000000000000000000070000000000DA
:103FE000000707070007000707070700000007078B
:103FF0000700000007070700000007070700000090
:104000000707070000070707070000070707070063
:104010000707000000000707070000000707070068
:104020000000070707000000070707000000070758
:10403000070000000707070000000707070000004F
:104040000000000007070000000007070000000054
:104050000707000000000707000000000707000036
:104060000000070700000000070700000000070726
:104070000000000000070000000000070000000032
:10408000000700000000000700000000000700001B
:10409000000000070000000000070000000000070B
:1040A00007070700070707070700070707070700B5
:1040B00000000707070007070707070007070707AC
:1040C0000700070707070700070707070700070795
:1040D000070707070007070707070007000000009A
:1040E000000707070707070007070707070707076E
:1040F000070707070000000007070000000000078F
:104100000707070000000707070700000707070762
:10411000070000070707070007000707070707074B
:104120000007070707070007070707070700070734
:10413000000000000707000000000707000000075C
:104140000707000000070707000000070707000037
:104150000007070700000007070707000707070712
:104160000700070707000700070707000700070702
:1041700007000007070707000007070707000007F9
:1041800007070707000707070707000707070707CD
:1041900007070700070707070700070707070700C4
:1041A00007070707070700070707070700070707AD
:1041B00007070007070707070007070707070007A4
:1041C00007000000000707000000000707000000CC
:1041D00000070700000000070707000000070707A7
:1041E000000000070707000000070707000000079E
:1041F0000007070700070007070700070007070772
:104200000007000707070007000707070007000768
:104210000707000700070707000700070707000751
:104220000707000000000707000000000707000064
:104230000000070700000000070700000000070754
:104240000000000007070000000007070000000052
:1042500007070700070707070700070707070707FC
:10426000000700070707070000000707070700000F
:1042700007070707000000070707000000000707FF
:1042800007070000000007070700000007070707EF
:1042900000000707070707070007070707070700CA
:1042A00007070707070700000000070707070707BA
:1042B00000000000000000000000000000000000FE
:1042C0000007070707070707070707070707070785
:1042D0000707070000000000000707070707070798
:1042E000000707070700070707070007070707007A
:1042F0000707070700070707070007070707000763
:104300000707070707070707070007070707000052
:104310000707070000070707070000070707000057
:104320000000070700000000070000000000000078
:10433000000000000000000000000000000000007D
:10434000070700070707070707000707070707070B
:104350000007070707070007000707070700000017
:10436000070707070000000707070000000007070E
:10437000070000000000070700000000070707070C
:1043800000000707070707070707070707070000D9
:1043900007070707070700000000070707070707C9
:1043A0000000000000000000000000070000000006
:1043B000070707070707070707070707070707078D
:1043C00007070700000000000007070707070707A7
:1043D0000707070700070707070700070707070082
:1043E0000707070700070707000007070707070772
:1043F0000707070707070707070007070707000062
:104400000707000000000707000000000707000082
:104410000000070000000000000000000000000095
:10442000000000000000000000000000000000008C
:104430000707070007070707070007070707070021
:10444000070707070700070707070700070707070A
:104450000700070707070707000007070707070701
:104460000000000000000000000000000700000045
:1044700000070707070007070707070707070707DA
:1044800007070707000000000000070707070707E6
:1044900007070700070707070700070707070007C1
:1044A00007070707000707070700070707070007B1
:1044B00007070700070707070700070707070000A8
:1044C000070007070707070007070700000007079F
:1044D0000700000707070700000707070007000796
:1044E000070700070007070700070007070700077F
:1044F0000000000000000707070707070707070776
:104500000707070707070707070707000000070750
:10451000000000000707000000000707000000007F
:104520000000000000070707070707000707070745
:104530000700070707070700000007070707000035
:104540000707070700000007070700000007070725
:10455000070707000007070707000007070707000E
:10456000000707070700000700070700000700070C
:1045700007070007000707070000000707070000FC
:1045800007070007070707070007070707070007D0
:1045900007070707000707070707070007070707B9
:1045A00007070007070707070700000707070707B0
:1045B00000000000000000000000000000000000FB
:1045C0000000070707070707070707070707070789
:1045D0000707070700000000000007070707070795
:1045E000000000070707000000070707000000079A
:1045F0000707070700070707070700070707070759
:104600000007070700000000070707070000000772
:10461000000707070000000707070000000707075B
:104620000000000707070707070007070707070736
:104630000007070707070700000007070707070726
:10464000000000000000000000000000000000006A
:104650000000070000000000070000000000070045
:104660000000000000000000000007000000000043
:104670000007070700070007070700070000000002
:10468000000000000000000000000000000000002A
:10469000000000000000000000000000000000001A
:1046A00007070000000007070000000000000000EE
:1046B00000000000000000000000000000000000FA
:1046C00000000000000000000000000000000000EA
:1046D0000707070707070000070707070000000094
:1046E00000000000000000000000000000000000CA
:1046F00000000000000000000000000000000000BA
:104700000707070707070707070707070000000055
:104710000000000000000000000000000000000099
:104720000000000000000000000000000000000089
:10473000070707000000070000000000000000005D
:104740000000000000000000000000000000000069
:104750000000000000000000000000000000000059
:104760000000000000070000000000000000000042
:104770000000000000000000000000000000000039
:104780000000000000000000000000000000000029
:1047900007070707070700070707070700000000CC
:1047A0000000000000000000000000000000000009
:1047B00000000000000000000000000000000000F9
:1047C00007070000000000000000000000000000DB
:1047D00000000000000000000000000000000000D9
:1047E00000000000000000000000000000000000C9
:1047F000000000000707000000000707000000009D
:1048000000000000000000000000000000000000A8
:104810000000000000000000000000000000000098
:10482000000707070000000707070000000000005E
:104830000000000000000000000000000000000078
:104840000000000000000000000000000000000068
:10485000070707070707070700070707000000000B
:104860000000000000000000000000000000000048
:104870000000000000000000000000000000000038
:104880000707000000000700000000000000000013
:104890000000000000000000000000000000000018
:1048A0000000000000000000000000000000000008
:1048B00000000007070700000007070700000000CE
:1048C00000000000000000000000000000000000E8
:1048D00000000000000000000000000000000000D8
:1048E000000007070707000000000707000000009E
:1048F00000000000000000000000000000000000B8
:1049000000000000000000000000000000000000A7
:104910000700000000000700000000000000000089
:104920000000000000000000000000000000000087
:104930000000000000000000000000000000000077
:104940000000000000000000000000000000000067
:104950000000000707070707000707070707000011
:104960000000000000000000000000000000000047
:104970000000000000000000000000000000000037
:1049800000000707070707000707070707000000E1
:104990000000000000000000000000000000000017
:1049A0000000000000000000000000000000000007
:1049B00000000004040404040004040404040000CF
:1049C00000000000000000000000000000000000E7
:1049D00000000000000000000000000000000000D7
:1049E000000004040404040004040404040000009F
:1049F00000000000000000000000000000000000B7
:104A000000000000000000000000000000000000A6
:104A10000000005F5F5F5F5F005FAFAFAFAF0000A0
:104A20000000000000000000000000000000000086
:104A30000000000000000000000000000000000076
:104A400000005F5F5F5F5F00AFAFAFAFAF00000020
:104A50000000000000000000000000000000000056
:104A60000000000000000000000C0C0C000CFF0C0B
:104A7000FF0C160CFF0CFFFF160CFF0C0C0C0016A5
:104A8000160C0C0C000000161616000000000000AA
:104A90000000000000000C0C0C000000FF0CFF0CDC
:104AA000FF00FFFFFF0CFF0C0C0C0C0CFF0C0C0CA0
:104AB0000C0C0C0016161600000000000000000090
:104AC0000002060000FB00FF0000F405030C0504D3
:104AD0000C05030C05040C05050000FF00FF000297
:104AE000090000F10400F900FF00010A0000E202E1
:104AF000010501010301010102050000FF0000CED4
:104B000002040404050000FF0000F100085A02043A
:104B10000302040402040502040602050000FF006B
:104B200001010007900000E208050000FF000208F4
:104B30000107C80106000100E700FF0001000007AF
:104B4000A00000EC0100FE00010100FF00010300D5
:104B500000E203010604010903050000FF00020151
:104B60000107C80106000100EC00FF00020400007C
:104B7000F10400F900FF0002010000F100FF000055
:104B8000ED00010602010100FF0000EC000102013E
:104B900007000207FF00010300FF0002080007648E
:104BA0000100140500F700FF0002090000F100FFFA
:104BB0000002040000F800085003084E03085402E5
:104BC000084C02085802084A01085C0000FC03086F
:104BD0006003085A03086003085A03086003085A70
:104BE00001050000FF0002040000FB00083E010375
:104BF0000201030201030201030201030201040A8C
:104C00000103020103020103020103020103020185
:104C10000402010302010302010302010302010372
:104C20000201040A0103020103020103020103025B
:104C30000103020104050103020103020103020151
:104C4000030201030201040501030201030201033F
:104C50000201030201030201040501030201030230
:104C600001030201030201030201050000FF00022B
:104C70000300085602040A0204080204060204049F
:104C800002040200084202030502040202030502B4
:104C900003050204020203050000F80403050404EE
:104CA00005040305040405040305040405040305C1
:104CB00001050000FF00077F0002020000FF00085E
:104CC0005701040E01040E01040E01040E01040E2E
:104CD00001040E01040E01040E01040E01040E0273
:104CE000076400084601040E01040E01040E0104CD
:104CF0000E01040E01040E01040E01040E01040E47
:104D000001040E02074600083C01040E01040E01D6
:104D1000040E01040E01040E01040E01040E010430
:104D20000E01040E01040E01050000FF000700043F
:104D300002040007FF000990000A3C0000FB010884
:104D400050030305030405030305030405030305DA
:104D50000304050303050304050303050304050316
:104D6000030503040503030503050000FF00070016
:104D70000402040007FF000990000A3C0000FB0148
:104D80000853030305030405030305030405030394
:104D900005030405030305030405030305030405D4
:104DA00003030503040503030503050000FF0007D3
:104DB000000402040007FF000990000A3C0000FB09
:104DC0000108560303050304050303050304050353
:104DD0000305030405030305030405030305030496
:104DE0000503030503040503030503050000FF0095
:104DF00007000402040007FF000990000A5A00009F
:104E0000FF01086303030503040503030503040509
:104E10000303050304050303050304050303050356
:104E2000040503030503040503030503050000FF50
:104E30000002020106000100E000FF00020101067D
:104E4000000100E000FF0002080106000100E00090
:104E5000FF0002050106000100E000FF0002090159
:104E600006000100E000FF000000C04A0000000052
:104E7000000000C84A00000000000000DC4A0000FA
:104E80000000000000DE4A00000000010000E94AC6
:104E900000000000000000FD4A00000000000000CB
:104EA000084B000000000100001F4B000000000044
:104EB00000002D4B000000000100003B4B000000F3
:104EC000000100004C4B000000000000005D4B00A2
:104ED0000000000000006B4B0000000000000076A6
:104EE0004B000000000100007E4B000000000100AC
:104EF00000894B000000000000009A4B00000000F9
:104F0000000000A84B00000000000000B04B0000B3
:104F10000000000000E54B000000000000006E4CA7
:104F200000000000000000B54C0000000000000080
:104F30002C4D000000000000006D4D00000000003E
:104F40000000AE4D00000000000000EF4D0000002A
:104F500000000000304E000000000000003B4E004A
:104F6000000000000000464E00000000000000515C
:104F70004E000000000000005C4E00000000112404
:104F80001FBECFEFD0E1DEBFCDBF1CE0A4E0B1E09B
:104F900001C01D92A53BB107E1F711E0A0E0B1E02F
:104FA000E6EEFEE802C005900D92A430B107D9F7F5
:104FB00014BE88E10FB6F8948093600010926000F0
:104FC0000FBEF89420E930E0F90185919491FC013D
:104FD000F07090832E5F3F4F80E0223C3807A1F7AE
:104FE0000E946D2B882311F40E944A2BEFEDF9E00B
:104FF00080E881939BE0EB3EF907D9F78FED99E0CC
:105000009093EC0B8093EB0B1092ED0B91E090934F
:10501000040C9093050C9093030C1092F00B1092DB
:10502000F60B1092FC0B1092020C1092C809109211
:10503000CA0982E18093C90980EE8093D00984E196
:105040008093CF091092D4091092D3091092D809F5
:105050001092D7099093EF0B0E94C03578940E946C
:1050600080350E948D360C9471470C94000030E01E
:105070003A95F1F731EC3A95F1F7C4E0D1E000EE62
:10508000A02E662776E02ED13BE23A95F1F70E94FA
:10509000702831E13A95F1F7AA9489F0C8956395A3
:1050A000683029F033E03A95F1F70000ECCF66273D
:1050B000002430E5C30FD01DC8950000E4CF35E0D3
:1050C0003A95F1F700C00ED1E091CA0942E0E42719
:1050D000E1FFE160E093CA09E2E0E0933600089561
:1050E000DE014D915D91679FC001480F591FFA0184
:1050F00028E2059108B94D91059108B95D91059196
:1051000008B900C0059108B9480F591F059108B9A1
:105110000591FA012A9508B961F7C895002708B9E1
:1051200008950F921F92EF93FF93FFB7E0918400D1
:10513000FF93E2FD04C0E1FD02C0000000C0E0FFFB
:1051400000C0E091C909EA95E093C909F091C80946
:10515000F0FD51C0EC3098F0F3E0F0938900FDE8E9
:10516000F0938800E0FB289826F4E1E00E94532A9F
:10517000B2C0E5E1EA95F1F70000289AACC0E6304C
:1051800008F100C000C02898E0FBE4E016F40E949B
:10519000532AE4E0E0933600E6E0E0936F009BC022
:1051A000EF93E0918400E2FD04C0E1FD02C0000045
:1051B00000C0E0FF00C0E2E00000289AE0936F002A
:1051C000EF91189500C0E0FB289826F4E1E00E94DA
:1051D000532A05C0E5E1EA95F1F70000289AE0912D
:1051E000C909E03009F077C0EDEFE093C909E1E0CB
:1051F000E093C80970C0E7E0E0938900EBE1E09339
:10520000880000C02898E2E000C00E94532AFDEF09
:105210000090CF09F019E091C909EF17D8F4FDEF1C
:105220000090CF09F0190090D009F019EF1790F015
:10523000EDE1FF2700800F92EA95E1F70FE10A9573
:10524000F1F700C00E943728E1E0FF270F9001929C
:10525000EE31E0F3E091C909E03009F03CC02F9352
:105260003F934F935F936F937F938F939F93AF93EE
:10527000BF9378941124EE27E093C809E2E1E0930C
:10528000C9098091D9099091DA0901968093D909C9
:105290009093DA09E091CB09F091CC09E115F10581
:1052A00009F009950E94392B0E94C1350E947D2981
:1052B0001124E091CD09F091CE09E115F10509F035
:1052C0000995BF91AF919F918F917F916F915F9160
:1052D0004F913F912F91EF91EFBFFF91EF911F9071
:1052E0000F9018952898E2E000C00E94532AE091A0
:1052F000C909EA95E093C9090895E091EF0BE0FD33
:105300000E94592C0090ED0B002019F4AFEDB9E08C
:1053100002C0A5EEBAE021E002260092ED0B22E0E9
:105320002093EE0BE091EF0BE0FF08952F923F9258
:105330004F925F926F927F928F929F92AF92BF92A5
:10534000CF92DF92EF92FF920F931F93CF93DF9351
:105350005091020C6091040C7091050C8091060C28
:105360002090F10B3090F20B4090F40B5090F50B25
:105370006090F30B1091F00B7090F70B8090F80B8E
:105380009090F90BA090FA0BB090FB0B2091F60BCC
:10539000C090FD0BD090FE0BE090000CF090010C43
:1053A0000091FF0B3091FC0B9FEF620C431CF2014C
:1053B000449141030008C12DD02D970CA81CF50184
:1053C000449142030008C10DD01D0C0DED1CF701E6
:1053D000449143030008C10DD01D8A956AF44091A1
:1053E000030C842F8695062E0694062600FA7695E1
:1053F000679576F940FF66F940E860FD4FE74503A1
:105400000008C10DD01D0024C038D0050CF0CFE736
:105410000A94C038D0050CF4C0E8C058CD939A95D2
:1054200009F0C3CF4091EE0B4A954093EE0B97E005
:1054300009F0BBCF6092F30B4092F40B9092F90B02
:10544000A092FA0B0093FF0BE092000C6093040C07
:105450007093050C8093060CDF91CF911F910F91F3
:10546000FF90EF90DF90CF90BF90AF909F908F9084
:105470007F906F905F904F903F902F900895E091B4
:10548000EB0BF091EC0B019100000093B3000BE0EB
:10549000EB3EF0070FED19E008F0F801E093EB0B9D
:1054A000F093EC0B08950F931F932F93EF93E091DC
:1054B000EB0BF091EC0B01910093B3000BE0EB3E92
:1054C000F0070FED19E008F0F801E093EB0BF09313
:1054D000EC0BE8E0EA95F1F7EF912F911F910F9116
:1054E000E0FD289AE0FF01C00895F4E1FA95F1F794
:1054F00000C0E1FD289AE1FF00C00895E0E6F4E075
:10550000A4E0B1E06091C4097091C5096D937D93E9
:105510003197E1F7112408959927552728E2220FA2
:10552000629F880F080E191EA4E0B1E0A00DB11D06
:105530006091C4097091C50920E3429F600D711DFF
:105540006D937C93112408959927772728E2220FE1
:10555000629F880F080E191EA4E0B1E0A00DB11DD6
:105560006091C6097091C70920E3429F600D711DCB
:10557000529F700D6D937C93112408958093C409FC
:105580009093C50908958093C6099093C70908951B
:105590008091CA09817008952091CA092E7F2093B5
:1055A000CA090895882329F48091D1099091D209DC
:1055B00008958091D5099091D6090895E0E6F0E02C
:1055C000808183FD089588E198E0F894808390833A
:1055D0007894FFCFF999FECF92BD81BD60BDF8945C
:1055E000FA9AF99A78940895F999FECF92BD81BDFF
:1055F000F894F89A80B5789408958093DC09909394
:10560000DD090895129AC895C895C895C89512984D
:1056100020E030E080E090E040E0369527959695D8
:105620008795C895C895C895C8951398009B30680C
:10563000019B9068139AC895C895C895C8954F5F07
:10564000403159F73093D2092093D1099093D6096C
:105650008093D5098091D1099091D2090F9731F0AB
:105660008091D5099091D6090F9711F40E94DE2AF6
:10567000089510920C0C009903C081E080930C0CEB
:10568000019905C080910C0C826080930C0C0E94E3
:10569000022B0895CF93DF93C0E0D0E0FE01E059E4
:1056A000FF4FE491CE016E2F0E94EA2A2196C0326C
:1056B000D105A1F7C0E2D0E0CE016FEF0E94EA2A47
:1056C000CE0101966FEF0E94EA2AA09688E0C030D2
:1056D000D80791F7DF91CF9108951F9380E090E074
:1056E0000E94F42A182F81E090E00E94F42A90E0B2
:1056F000382F20E0210F311D2A55354509F491E05E
:10570000892F1F910895FC016787089581E091E03A
:105710009093050C8093040C6093030C0895FC0196
:1057200082810E94712F0895FC018181680F61833D
:1057300082810E945A2F0895FC01862F6181681B87
:10574000618382810E945A2F0895FC0180818F75A8
:1057500080830895FC018081806480830895FC012A
:1057600066870895FF920F931F938C01F62EFC011C
:1057700082810E945A2FF801F1828081877F808385
:105780001F910F91FF900895FC0162870895FC011D
:1057900063870895CF93DF93EC01462F898190E0D2
:1057A000FC01EE0FFF1FE45EF04A25913491E62FD5
:1057B000FF27E7FDF095E80FF91FEE0FFF1FE45EEE
:1057C000F04A859194916885821B930B70E00E944A
:1057D0006A469B016115710511F421E030E08A8170
:1057E00090E0FC01EE0FFF1FE80FF91FEE0FFF1F07
:1057F000E051F44F81819281820F931F92838183C4
:105800003E832D838881886088838981840F8F837C
:10581000DF91CF910895FC0160870895FC016483B6
:105820000895DC0114968C911497882331F15596D4
:10583000ED91FC915697662371F0262F332727FDB3
:10584000309520953095C901880F991F820F931FBD
:10585000E80FF91F08C033973297849132968D3044
:1058600011F08F3FC1F75696FC93EE93559714961F
:105870008C911497815014968C93089590936E0C8C
:1058800080936D0C8FE68093700C1092DE09EFE030
:10589000FCE080E090E13FEF28E182839083158671
:1058A0003487108A238790878F5F77968430A9F793
:1058B0000895A0E0B0E0EFE5FCE20C94A946AFE06B
:1058C000BCE0C1EFDBE01F968C911F978823B9F0F5
:1058D000282F332727FD30951E968C911E97280F71
:1058E000311D2F3F310519F014F02FEF30E0C901C1
:1058F00037FF02C080E090E01E968C931E978C913B
:1059000083FF26C015964D915C91169728813981A9
:10591000240F351F3983288317968C911797E82F0A
:10592000F0E0EE0FFF1FE45EF04A859194911416AB
:10593000150624F42817390730F40AC0452B41F026
:105940008217930728F0998388838C91877F8C93A3
:10595000579626964CE0AB36B40709F0B4CF809149
:10596000DE09882309F0DEC0F1C0E091740CF091EB
:10597000750CCF0101969093750C8093740C449133
:105980004F3F69F5AC014F5F5F4F5093750C4093EB
:10599000740CFC0184918F3219F41092DE09D0C08E
:1059A000863009F0B2C0FA013196CF01019690938A
:1059B000750C8093740CE491E33529F49093770C83
:1059C0008093760CA2C0E53409F09FC08091760CDC
:1059D0009091770C9093750C8093740C96C047FF50
:1059E00002C040936F0C20916F0C322F3F7047FF25
:1059F00008C001969093750C8093740C0197FC017C
:105A00004491822F90E0807F9070803B910531F12E
:105A1000803C910509F46DC08039910509F075C08D
:105A2000E091740CF091750C3196F093750CE09345
:105A3000740C3197E491832F90E08C9FD0018D9F5F
:105A4000B00D9C9FB00D1124A15FB34FEE0F832FBB
:105A500050966C912E2F0E94332F57C0E091740CFA
:105A6000F091750C3196F093750CE093740C3197AE
:105A70002491473071F4832F90E08C9FF0018D9F2B
:105A8000F00D9C9FF00D1124E15FF34F220F24874E
:105A90003CC04B3071F4832F90E08C9FF0018D9FC0
:105AA000F00D9C9FF00D1124E15FF34F220F238333
:105AB0002CC04C3571F4832F90E08C9FF0018D9FAA
:105AC000F00D9C9FF00D1124E15FF34F220F228710
:105AD0001CC04436D1F4832F90E08C9FF0018D9F41
:105AE000F00D9C9FF00D1124E15FF34F220F2387EF
:105AF0000CC0832F90E08C9FF0018D9FF00D9C9F38
:105B0000F00D1124E15FF34F408B84E79CE00E948D
:105B1000702E9093720C8093710C10926C0C1092FA
:105B20006B0C02C0C7E1D0E020916B0C30916C0C83
:105B30008091710C9091720C2817390709F415CFD8
:105B40002F5F3F4F30936C0C20936B0CCFE0DCE069
:105B500000EF1BE08FEFC82ED12C7E018881282F0B
:105B600085FF39C08D899E89892B09F434C026FFB1
:105B70002BC031C0ED89FE89CF0101969E8B8D8BA4
:105B800024912F3F31F488818F7788831E8A1D8A64
:105B90001FC001969E8B8D8B0197FC016491822F13
:105BA00090E0880F991F8E539F4FFC0125913491EF
:105BB000C701F9010995ED89FE893196FE8BED8BC0
:105BC0003197E491EA8B1B8A9B898A89981791F215
:105BD0008B898F5F8B8B888185FD03C020E030E04F
:105BE00070C08C898F3F11F08F5F8C8B888187FF0D
:105BF00002C08FEF01C08C859D85992309F45BC09D
:105C00002E85222309F457C0882309F454C04091FB
:105C1000700C442309F44FC0899FC00111248050A7
:105C20009F4F892F992730E0B901869F9001879F68
:105C3000300D969F300D112420503F4F232F3327D6
:105C40008B8190E0FC012E9FC0012F9F900D3E9F05
:105C5000900D112480509F4F892F9927242F30E0D9
:105C6000AC01429FC001439F900D529F900D1124A3
:105C700080509F4F292F33278A858823F1F0E985AB
:105C8000F0E0E050FF49E491E058E89FC0011124A2
:105C900080509F4F892F9927B601681B790B629F0F
:105CA000C001639F900D729F900D112480509F4FF3
:105CB000292F332702C020E030E089859B85890F9A
:105CC0008987F801208367960A5F1F4FFCE0CB3677
:105CD000DF0709F042CFCDB7DEB7E8E00C94C54648
:105CE000DC01ED91FC911197AF014F5F5F4F119671
:105CF0005C934E93E4912E2F30E0E7FF13C02F7793
:105D000030703695322F222737952795FA014F5F4D
:105D10005F4FE4918E2F8F77280F311DE7FDF1CF74
:105D20004D935C93C90108950F931F93CF93DF9315
:105D3000EC01062F10E0888187FD11E01F869FEFA0
:105D40009E874D871C8A8881877B88831A8619865F
:105D500029831C829B838A81833069F4112309F48F
:105D6000022F81E091E09093050C8093040C81E078
:105D70008093030C07C0622F0E945A2F8A8160E033
:105D80000E94712F112311F0098B01C0088B89E04B
:105D9000089FC0011124E0916D0CF0916E0CE80F8A
:105DA000F91F3396259134912115310519F41E8A76
:105DB0001D8A08C01B8AF90184918A8B2F5F3F4F8F
:105DC0003E8B2D8BDF91CF911F910F9108950F93F3
:105DD0001F93282F362F89E0289FC0011124E091BE
:105DE0006D0CF0916E0CE80FF91F8491813011F465
:105DF00083E021C0823011F484E01DC08091260C24
:105E000087FF16C08091370C821711F4442381F468
:105E100080913D0C87FF0EC080914E0C821711F4CB
:105E2000442341F490913A0C8091510C891710F45D
:105E300081E001C082E007E1809F80011124015FC1
:105E4000134F80E8F8018083168A158AC801622FF3
:105E5000432F20E50E94942EF80180818062808388
:105E60001F910F910895CF93DF93342F97E1899F6E
:105E7000E0011124C15FD34F8881982F85FF02C0B4
:105E800087FD15C0222341F48F85882311F496FFE6
:105E90001D8688818F7B0AC018821E8A1D8ACE01CA
:105EA000422F232F0E94942E888180628883DF9165
:105EB000CF91089599277727833008F00895ECE172
:105EC000FFE5660F771FE60FF71FA591B491E0EF8E
:105ED000FBE026E0289FE00DF11DA183B283112491
:105EE000089599277727E0EFFBE026E0289FE00D53
:105EF000F11D6E3F31F46091030C6E7F6093030CD3
:105F00000BC06F3F31F46091030C6E6F6093030C14
:105F100003C071E6760F75831124089522002400D2
:105F2000260028002B002D003000330036003900F9
:105F30003D004000440048004C00510056005B000A
:105F4000600066006C00730079008100880090009A
:105F50009900A200AC00B600C100CC00D800E5005A
:105F6000F3000101100121013201440157016C01CC
:105F700081019801B001CA01E5010202210241023A
:105F800064028802AE02D702030330036103940364
:105F9000CB03050442048304C70410055D05AF0567
:105FA00005066106C2062907960709088308050940
:105FB0008E09200ABA0A5D0B0A0CC10C840D510E21
:105FC0002B0F121007110A121D1340147415BA1664
:105FD00014188319071BA31C571E24200E221424F7
:105FE00039267F28E82A752D293006330F364539A2
:105FF000AD3C49401B442848734CFE50CF55EA5AEB
:1060000051600C661D6C8B725A7992803788509063
:10601000E598FDA19FABD3B5A3C000000000000030
:106020000000000000000000000000000000000070
:106030000000000000000000000000000000000060
:106040000000000000000000000000000000000050
:106050000000000000000000000000000000000040
:106060000000000000000000000000000000000030
:106070000000000000000000000000000000000020
:106080000000000000000000000000000000000010
:106090000000000000000000000000000000000000
:1060A00000000000000000000000000000000000F0
:1060B00000000000000000000000000000000000E0
:1060C00000000000000000000000000000000000D0
:1060D00000000000000000000000000000000000C0
:1060E00000000000000000000000000000000000B0
:1060F00000000000000000000000000000000000A0
:10610000000306090C101316191C1F2225282B2E1C
:10611000313336393C3F414447494C4E5153555831
:106120005A5C5E60626466686A6B6D6F70717374EE
:10613000757678797A7A7B7C7D7D7E7E7E7F7F7FA7
:106140007F7F7F7F7E7E7E7D7D7C7B7A7A7978768D
:1061500075747371706F6D6B6A68666462605E5CA3
:106160005A585553514E4C494744413F3C393633B8
:10617000312E2B2825221F1C191613100C0906037B
:1061800000FDFAF7F4F0EDEAE7E4E1DEDBD8D5D282
:10619000CFCDCAC7C4C1BFBCB9B7B4B2AFADABA84D
:1061A000A6A4A2A09E9C9A9896959391908F8D8C70
:1061B0008B8A888786868584838382828281818197
:1061C0008181818182828283838485868687888A91
:1061D0008B8C8D8F9091939596989A9C9EA0A2A45B
:1061E000A6A8ABADAFB2B4B7B9BCBFC1C4C7CACD26
:1061F000CFD2D5D8DBDEE1E4E7EAEDF0F4F7FAFD43
:10620000808182838485868788898A8B8C8D8E8F16
:10621000909192939495969798999A9B9C9D9E9F06
:10622000A0A1A2A3A4A5A6A7A8A9AAABACADAEAFF6
:10623000B0B1B2B3B4B5B6B7B8B9BABBBCBDBEBFE6
:10624000C0C1C2C3C4C5C6C7C8C9CACBCCCDCECFD6
:10625000D0D1D2D3D4D5D6D7D8D9DADBDCDDDEDFC6
:10626000E0E1E2E3E4E5E6E7E8E9EAEBECEDEEEFB6
:10627000F0F1F2F3F4F5F6F7F8F9FAFBFCFDFEFFA6
:10628000000102030405060708090A0B0C0D0E0F96
:10629000101112131415161718191A1B1C1D1E1F86
:1062A000202122232425262728292A2B2C2D2E2F76
:1062B000303132333435363738393A3B3C3D3E3F66
:1062C000404142434445464748494A4B4C4D4E4F56
:1062D000505152535455565758595A5B5C5D5E5F46
:1062E000606162636465666768696A6B6C6D6E6F36
:1062F000707172737475767778797A7B7C7D7E7F26
:1063000000020406080A0C0E10121416181A1C1E9D
:1063100020222426282A2C2E30323436383A3C3E8D
:1063200040424446484A4C4E50525456585A5C5E7D
:1063300060626466686A6C6E70727476787A7C7E6D
:106340007F7D7B79777573716F6D6B69676563614D
:106350005F5D5B59575553514F4D4B49474543413D
:106360003F3D3B39373533312F2D2B29272523212D
:106370001F1D1B19171513110F0D0B09070503011D
:10638000FFFDFBF9F7F5F3F1EFEDEBE9E7E5E3E10D
:10639000DFDDDBD9D7D5D3D1CFCDCBC9C7C5C3C1FD
:1063A000BFBDBBB9B7B5B3B1AFADABA9A7A5A3A1ED
:1063B0009F9D9B99979593918F8D8B8987858381DD
:1063C00080828486888A8C8E90929496989A9C9EDD
:1063D000A0A2A4A6A8AAACAEB0B2B4B6B8BABCBECD
:1063E000C0C2C4C6C8CACCCED0D2D4D6D8DADCDEBD
:1063F000E0E2E4E6E8EAECEEF0F2F4F6F8FAFCFEAD
:106400007F7F7F7F7F7F7F7F7F7F7F7F7F7F7F7F9C
:106410007F7F7F7F7F7F7F7F7F7F7F7F7F7F7F7F8C
:106420007F7F7F7F7F7F7F7F7F7F7F7F7F7F7F7F7C
:106430007F7F7F7F7F7F7F7F7F7F7F7F7F7F7F7F6C
:106700000309131E28313A40464C5054585B5E61D1
:10671000636567696B6C6E6F707172737475767791
:10672000777879797A7A7B7B7C7C7C7D7D7D7E7EB7
:106730007E7E7F7F7F7F7F7F7F7F7F7F7F7F7F7F6B
:106740007F7F7F7F7F7F7F7F7F7F7F7F7F7E7E7E5C
:106750007E7D7D7D7C7C7C7B7B7A7A79797877778E
:10676000767574737271706F6E6C6B696765636157
:106770005E5B5854504C46403A31281E13090300C2
:10678000C6CCD5DBDFE3E5E7E9EAEBECEDEEEFEFD6
:10679000F0F0F0F1F1F1F1F2F2F2F2F2F2F2F2F3E2
:1067A000F3F3F3F3F3F3F3F3F3F3F3F3F3F3F3F3B9
:1067B000F3F3F3F3F3F3F3F3F3F3F3F3F3F3F3F3A9
:1067C000F3F3F3F3F3F3F3F3F3F3F3F3F3F3F3F399
:1067D000F3F3F3F3F3F3F3F3F3F3F3F3F3F3F3F389
:1067E000F2F2F2F2F2F2F2F2F1F1F1F1F0F0F0EF96
:1067F000EFEEEDECEBEAE9E7E5E3DFDBD5CCC60055
:1068000000283D42302D2C2B2C2D2E2F30323335AD
:1068100037393B3D3F414345484A4C4E505355570D
:10682000595B5D5F61636567696B6C6E70717374F2
:10683000757778797A7B7C7D7D7E7E7F7F7F7F7F99
:106840007F7F7F7F7F7F7E7E7D7D7C7B7A7978777F
:1068500075747371706E6C6B69676563615F5D5BA6
:1068600059575553504E4C4A484543413F3D3B399B
:1068700037353332302F2E2D2C2B2C2D30423D2806
:1068800000E9E5FED4D7D7D7D6D4D2D0CECCCAC86B
:10689000C6C3C1BFBDBAB8B6B4B1AFADABA9A7A5A9
:1068A000A3A19F9E9C9A999795949391908F8D8C7C
:1068B0008B8A89888887868585848484838383837B
:1068C0008383838383848484858586878888898A73
:1068D0008B8C8D8F909193949597999A9C9E9FA164
:1068E000A3A5A7A9ABADAFB1B4B6B8BABDBFC1C37C
:1068F000C6C8CACCCED0D2D4D6D7D7D7D4FEE5E935
:10690000F9F8F9F5EBE1DDDEE0E2E4E5E6E5E4E205
:10691000DED9D2CAC1B7ACA299918A868381808020
:106920008182838586888A8C8D8F909293959697A5
:1069300098999A9B9B9C9D9D9D9E9E9E9F9F9F9F8D
:106940009F9F9F9E9E9E9D9D9D9C9B9B9A99989785
:1069500096959392908F8D8C8A888685838281808C
:10696000808183868A9199A2ACB7C1CAD2D9DEE26E
:10697000E4E5E6E5E4E2E0DEDDE1EBF5F9F8F90077
:106980000708070B151F2322201E1C1B1A1B1C1E89
:1069900022272E363F49545E676F767A7E7F7F7F4F
:1069A0007F7E7D7B7A7876747371706E6D6B6A69A9
:1069B00068676665656464636362626261616161A0
:1069C0006161616262626363636465656667686989
:1069D0006A6B6D6E7071737476787A7B7D7E7F7F63
:1069E0007F7F7E7A766F675E54493F362E27221E60
:1069F0001C1B1A1B1C1E2022231F150B0708070037
:106A00001F313D444E5354565A5F64696E74767913
:106A10007C7F7F7F7F7F7F7F7F7F7F7F7F7F7F7F89
:106A20007F7F7F7F7F7F7F7F7F7F7F7F7F7F7F7F76
:106A30007F7F7F7F7F7F7F7F7F7F7F7F7F7F7F7F66
:106A40007F7F7F7F7F7F7F7F7F7F7F7F7F7F7F7F56
:106A50007F7F7F7F7F7F7F7F7F7F7F7F7F7F7F7F46
:106A60007F7F7F7F7F7F7F7F7F7F7F7F7F7F7F7F36
:106A70007F7F7F7F7F7F7F7F7F7F7F7C7871684C88
:106A80002C1C120C0A0B0A05FDF3E9DFD4CAC0B7AF
:106A9000AEA69E97918B8685828080808080808044
:106AA00080808080808080808080808080808080E6
:106AB00080808080808080808080808080808080D6
:106AC00080808080808080808080808080808080C6
:106AD00080808080808080808080808080808080B6
:106AE00080808080808080808080808080808080A6
:106AF000808080808087919DACC4CBD4DDF2FAFA8F
:106B00000F931F9387EF90E00E943E2C00E011E06E
:106B1000C8010E94C32AC8010E94BE2A0E947E2A80
:106B20008FE090E00E94523680E06FEF41E00E94DB
:106B3000E72E00E518E082E16CE0A8010E94C43570
:106B400083E090E00E94523682E16CE044E858E035
:106B50000E94C43582E090E00E94523682E16CE0EF
:106B6000A8010E94C43580E290E00E9452360E9443
:106B70007E2A8AE090E00E9452361F910F9108957C
:106B800008950E9469360895A0E0B0E0EAECF5E3CC
:106B90000C94A446782E862EEA01FA01C590D49072
:106BA000FA013296A590B49000E016C0FC01EE0DFB
:106BB000FF1D3296EE0FFF1FEC0FFD1F4591549104
:106BC000812F870D692D0E94A42A1F5F812F90E0DD
:106BD0008C159D055CF30F5F802F90E08A159B0557
:106BE0005CF48C9D70018D9DF00C9C9DF00C11242B
:106BF00010E0902E980CEACFCDB7DEB7EDE00C9404
:106C0000C046EF92FF920F931F93CF93DF93F62E20
:106C1000042FE22EEC0110E0002311F4112349F4BB
:106C2000802F6AE00E944A46905F8C2F6F2D492F7B
:106C300009C0EE2021F08C2F6F2D40E103C08C2F76
:106C40006F2D40E00E948C2A1F5F2197133031F096
:106C5000802F6AE00E944A46082FDECFCDB7DEB70C
:106C6000E6E00C94C746FF920F931F93CF93DF93F8
:106C70008C01F62EEA01FE0144912196442349F04D
:106C8000802F0F5F1F4F4F7740526F2D0E948C2A2D
:106C9000F2CFCDB7DEB7E5E00C94C84640520E9473
:106CA0008C2A08950F931F93CF93DF938C01C0E03C
:106CB000D0E007C00E94C82A8823E1F30E94CC2AB2
:106CC0002196C017D107B4F3DF91CF911F910F9197
:106CD000089580917B0C8823F9F080917C0C8823A7
:106CE000C1F48091790C80937C0C80917D0CE82F0D
:106CF000F0E0E555F74FE491E7B990917A0C980FE1
:106D000090937D0C992311F09D3031F410927B0CFF
:106D10000895815080937C0C0895A0E0B0E0E3E9F1
:106D2000F6E30C94AA4687E69EE40E943E2C84E09B
:106D30009AE00E94BE2A80E79CE10E94C32A88EA6A
:106D400095E10E94FD2A0E94E0376091930C615FFB
:106D50008BE045EF50E00E94A42A6091930C615FA4
:106D60008CE046EF50E00E94A42A6091930C615F92
:106D70008BE145EF50E00E94A42A6091930C615F83
:106D80008CE146EF50E00E94A42A92E0D92E809137
:106D90000A0C90910B0C0D9690930B0C80930A0C9F
:106DA00080E00E94D22AEC0180918B0C882341F470
:106DB00085E190E060E170E04DEE59E00E943336ED
:106DC00080918B0C813041F485E190E060E170E0CE
:106DD00041EF59E00E9433368091940C882341F4AE
:106DE00085E190E061E170E045EF59E00E943336C3
:106DF0008091940C813041F485E190E061E170E094
:106E00004AEF59E00E9433368091940C823041F46D
:106E100085E190E061E170E04FEF59E00E94333688
:106E2000CE0188709170892B21F4C0FD02C0C2FF91
:106E300011C080E00E94D22A892BD9F78091930C4F
:106E4000882341F40E94203880910A0C90910B0C09
:106E50000E942C47CE0180739070892B09F464C086
:106E60006091930C615F8BE042E150E00E94A42AA4
:106E70006091930C615F8CE042E150E00E94A42A93
:106E80006091930C615F8BE142E150E00E94A42A83
:106E90006091930C615F8CE142E150E00E94A42A72
:106EA00081E060E941E00E94E72EC4FF09C08091C3
:106EB000930C882319F4D092930C11C081500DC00B
:106EC000CE0184729070892B51F08091930C8230A6
:106ED00019F41092930C03C08F5F8093930C609110
:106EE000930C615F8BE045EF50E00E94A42A609113
:106EF000930C615F8CE046EF50E00E94A42A609101
:106F0000930C615F8BE145EF50E00E94A42A6091F1
:106F1000930C615F8CE146EF50E00E94A42A80E070
:106F20000E94D22A892BD9F78E010074107080E854
:106F3000E82EF12CEC22FD229E01207C09F427CFC3
:106F40008AE060E941E00E94E72E9091930C913035
:106F5000C1F4012B49F080918B0C882319F4909394
:106F60008B0C28C081500AC0EF2821F180918B0C36
:106F7000813019F410928B0C1DC08F5F80938B0CA5
:106F800019C09230B9F4012B49F08091940C8823F8
:106F900019F49093940C0EC081500AC0EF2851F060
:106FA0008091940C823019F41092940C03C08F5F7E
:106FB0008093940C80E00E94D22A892BD9F7E7CEE7
:106FC0000E947E2A81E190E06FE070E049ED59E097
:106FD0000E9433368FE090E060E170E04FED59E0C1
:106FE0000E9433368FE090E061E170E046EE59E0B8
:106FF0000E94333689E090E066E170E04CE50E9443
:107000004E368BE090E066E170E044EC59E00E947F
:10701000333685E190E060E170E04DEE59E00E948A
:10702000333685E190E061E170E045EF59E00E9480
:10703000333682E063E048E05AE10E94C4350895A7
:1070400080918B0C882329F489E160E941E00E945A
:10705000E72E0E947E2A80E065E044EA55E10E9426
:10706000C43588E790E09093AF0C8093AE0C81E03C
:1070700090E00E9478380E94C93A0E9410390E941C
:10708000FD3B8091AE0C9091AF0C892B11F40E94C6
:107090001D458091820C9091830C8135910511F4EE
:1070A0000E94693B8091800C9091810C0196909395
:1070B000810C8093800C8091900C9091910C0196A2
:1070C0009093910C8093900C44976CF01092910CDB
:1070D0001092900C8091AE0C9091AF0C0197909310
:1070E000AF0C8093AE0C81E090E00E945236C3CF8B
:1070F0001F93182F0E947E2A80E065E044EA55E144
:107100000E94C435113009F51093A30C24E130E03E
:107110003093890C2093880C81E090E09093830C4D
:107120008093820C3093870C2093860C8AE090E049
:107130009093AB0C8093AA0C90E08091A50C8823CF
:1071400009F491E09093A50C1BC01230C9F481E0C2
:107150008093A30C24E130E03093890C2093880CB9
:1071600081E090E09093830C8093820C3093870CA5
:107170002093860C8AE090E09093AB0C8093AA0C4D
:107180002BE02093A20C82E080937E0C89E0809318
:10719000950C8091A50C8823D9F090E19093B40CC4
:1071A00088E08093B00C9093850C20937F0C909393
:1071B000A70C8EE08093920C83E18093A60C209321
:1071C000A90C8CE18093970C2093B30C87E01AC034
:1071D00096E19093B40C88E08093B00C9093850C6A
:1071E00020937F0C9093A70C8EE08093920C83E108
:1071F0008093A60C2093A90C8AE08093970C20938F
:10720000B30C8FE180938A0C8AE090E00E945236A2
:107210000E94C03B0E94C93A0E94FD3B1F91089505
:107220001F9380E00E94D22A182F90918A0C80919F
:10723000B40C981741F49091A20C8091B00C98175F
:1072400011F40E94204490918A0C8091850C98172B
:1072500041F49091A20C80917F0C981711F40E9438
:10726000204490918A0C8091A70C981741F490913A
:10727000A20C8091920C981711F40E9420449091D6
:107280008A0C8091A60C981741F49091A20C8091E1
:10729000A90C981711F40E94204490918A0C8091B7
:1072A000970C981741F49091A20C8091B30C981709
:1072B00011F40E94204414FF26C080E00E94D22ACC
:1072C000892BD9F76091A20C6930ECF06350609380
:1072D000A20C6D5F80918A0C42E150E00E94A42ACA
:1072E00080918A0C6091A20C6D5F8F5F42E150E04B
:1072F0000E94A42A80918B0C882329F485E060E900
:1073000041E00E94E72E15FF26C080E00E94D22AAD
:10731000892BD9F76091A20C6C30ECF46D5F60930F
:10732000A20C635080918A0C42E150E00E94A42A92
:1073300080918A0C6091A20C63508F5F42E150E013
:107340000E94A42A80918B0C882329F485E060E9AF
:1073500041E00E94E72E8091A50C882309F49FC08C
:1073600017FF13C180E00E94D22A892BD9F7209100
:107370008A0C203224F58091820C9091830C803508
:107380009105E9F02D5F20938A0C2350822F6091A4
:10739000A20C42E150E00E94A42A80918A0C825003
:1073A0006091A20C42E150E00E94A42A80918B0CD3
:1073B000882329F485E060E941E00E94E72E80916E
:1073C000820C9091830C813591052CF40196909359
:1073D000830C8093820C2091880C3091890C2F5F54
:1073E0003F4F3093890C2093880C40918A0C8091F8
:1073F000B40C481731F49091A20C8091B00C9817FE
:1074000099F18091850C481731F49091A20C8091EC
:107410007F0C981749F18091A70C481731F490918F
:10742000A20C8091920C9817F9F08091A60C481745
:1074300031F49091A20C8091A90C9817A9F0809139
:10744000970C481731F49091A20C8091B30C9817C7
:1074500059F08091AA0C9091AB0C009729F00197FC
:107460009093AB0C8093AA0C233331053CF43093FA
:10747000870C2093860C2233310544F084E690E09B
:10748000821B930B9093870C8093860C423209F0F9
:107490007CC087E080938A0C10928D0C76C016FF1A
:1074A00074C080E00E94D22A892BD9F720918A0CDF
:1074B000273091F48FE180938A0C87E06091A20CD1
:1074C00042E150E00E94A42A88E06091A20C42E1CF
:1074D00050E00E94A42A26C0283024F18091820C1A
:1074E0009091830C80359105E9F0235020938A0C0C
:1074F0002D5F822F6091A20C42E150E00E94A42AED
:1075000080918A0C8C5F6091A20C42E150E00E9455
:10751000A42A80918B0C882329F485E060E941E05E
:107520000E94E72E8091820C9091830C8135910509
:107530002CF401969093830C8093820C2091880CFC
:107540003091890C2F5F3F4F3093890C2093880C2A
:107550008091AA0C9091AB0C009729F00197909321
:10756000AB0C8093AA0C233331053CF43093870C89
:107570002093860C2233310544F084E690E0821B90
:10758000930B9093870C8093860C0E94C03B1F91B5
:10759000089581E090E060E070E048EB58E00E94E0
:1075A000333683E090E061E070E04091A30C20E08E
:1075B0000E9401368EE090E060E070E04DEB58E014
:1075C0000E94333682E190E061E070E04091880CE7
:1075D00020E00E9401368091A50C2091880C30910A
:1075E000890C8823C1F02233310544F483E190E013
:1075F00061E070E045EE58E00E9433368091880CDF
:107600009091890CC39704F183E190E061E070E010
:1076100048EE58E017C02233310544F483E190E08E
:1076200061E070E048EE58E00E9433368091880CAB
:107630009091890CC39744F083E190E061E070E0A1
:1076400045EE58E00E9433368DE190E060E070E056
:1076500048EC58E00E94333682E290E061E070E04E
:107660004091AA0C20E00E94013681E190E064E0A4
:1076700070E043ED58E00E94333683E190E063E030
:1076800070E04091AE0C20E00E94013681E090E075
:1076900064E070E048ED58E00E9433368FE190E0FE
:1076A00064E070E04DED58E00E94333683E090E0F6
:1076B00063E070E040918E0C20E00E94013682E28F
:1076C00090E063E070E04091980C20E00E94013669
:1076D00008958AE090E06BE070E04BEE58E00E9485
:1076E000333680918B0C882329F489E160E941E0ED
:1076F0000E94E72E80E00E94D22A83FFFBCF80E029
:107700000E94D22A892BD9F78091A50C882351F0A9
:1077100080918E0C90918F0C069690938F0C809395
:107720008E0C09C08091980C9091990C06969093BC
:10773000990C8093980C0E94274764E070E00E94A7
:107740006A468093960C8130B9F48091A50C882309
:1077500051F080918E0C90918F0C019690938F0C2C
:1077600080938E0C09C08091980C9091990C019691
:107770009093990C8093980C81E00E94783808953A
:1077800080918A0C6091A20C4FEE50E00E94A42AD6
:1077900080918A0C8F5F6091A20C40EF50E00E94B4
:1077A000A42A8091800C9091810C64E070E00E948A
:1077B0006A46029784F480918A0C6091A20C4FEE85
:1077C00050E00E94A42A80918A0C8F5F6091A20CE5
:1077D00040EF50E00FC080918A0C6091A20C43EF03
:1077E00050E00E94A42A80918A0C8F5F6091A20CC5
:1077F00044EF50E00E94A42A08958091B40C609157
:10780000B00C41EF50E00E94A42A8091B40C8F5F2D
:107810006091B00C42EF50E00E94A42A8091850C48
:1078200060917F0C41EF50E00E94A42A8091850C6A
:107830008F5F60917F0C42EF50E00E94A42A8091FC
:10784000A70C6091920C41EF50E00E94A42A809115
:10785000A70C8F5F6091920C42EF50E00E94A42A27
:107860008091A60C6091A90C41EF50E00E94A42ADF
:107870008091A60C8F5F6091A90C42EF50E00E94AE
:10788000A42A8091970C6091B30C41EF50E00E94C4
:10789000A42A8091970C8F5F6091B30C42EF50E067
:1078A0000E94A42A80918B0C882341F50E942747CF
:1078B00062E870E00E946A4680938C0C0E94274721
:1078C00061E970E00E946A468093AD0C0E942747F0
:1078D00065EA70E00E946A468093B20C0E942747D6
:1078E00068E770E00E946A468093A40C0E942747D4
:1078F0006EE670E00E946A468093840C80918B0C47
:10790000813041F50E94274764E670E00E946A4694
:1079100080938C0C0E94274763E770E00E946A46C0
:107920008093AD0C0E94274767E870E00E946A468A
:107930008093B20C0E9427476AE570E00E946A4675
:107940008093A40C0E94274760E570E00E946A467D
:107950008093840C80918B0C823041F50E942747E4
:1079600060E570E00E946A4680938C0C0E94274775
:107970006FE570E00E946A468093AD0C0E94274735
:1079800063E770E00E946A468093B20C0E9427472A
:1079900066E470E00E946A468093A40C0E94274728
:1079A0006CE370E00E946A468093840C80918C0C9A
:1079B000813009F070C14091B40C80918A0C841719
:1079C0000CF055C0242F332727FD3095235030402D
:1079D0008091850C992787FD90952817390739F4F0
:1079E0009091B00C80917F0C981709F440C0809161
:1079F000A70C992787FD90952817390731F49091A6
:107A0000B00C8091920C981791F18091A60C992757
:107A100087FD90952817390731F49091B00C80912B
:107A2000A90C981721F18091970C992787FD9095C3
:107A30002817390731F49091B00C8091B30C981746
:107A4000B1F04830A4F043504093B40C4D5F842F04
:107A50006091B00C42E150E00E94A42A8091B40CE5
:107A60008C5F6091B00C42E150E00E94A42A4091EA
:107A7000B40C80918A0C48170CF055C0242F332782
:107A800027FD30952D5F3F4F8091850C992787FD0D
:107A900090952817390739F49091B00C80917F0C9C
:107AA000981709F440C08091A70C992787FD9095FD
:107AB0002817390731F49091B00C8091920C9817E7
:107AC00091F18091A60C992787FD90952817390789
:107AD00031F49091B00C8091A90C981721F180910C
:107AE000970C992787FD90952817390731F49091C5
:107AF000B00C8091B30C9817B1F04032A4F44D5FF4
:107B00004093B40C4350842F6091B00C42E150E09C
:107B10000E94A42A8091B40C82506091B00C42E182
:107B200050E00E94A42A6091B00C8091A20C8617AC
:107B30000CF055C0262F332727FD309523503040B9
:107B400080917F0C992787FD90952817390739F484
:107B50009091B40C8091850C981709F440C08091E5
:107B6000920C992787FD90952817390731F4909149
:107B7000B40C8091A70C981791F18091A90C9927CA
:107B800087FD90952817390731F49091B40C8091B6
:107B9000A60C981721F18091B30C992787FD909539
:107BA0002817390731F49091B40C8091970C9817ED
:107BB000B1F06930A4F063506093B00C6D5F8091B8
:107BC000B40C42E150E00E94A42A8091B40C609170
:107BD000B00C6D5F8F5F42E150E00E94A42A60917B
:107BE000B00C8091A20C68170CF055C0262F3327DB
:107BF00027FD30952F5F3F4F80917F0C992787FDA0
:107C000090952817390739F49091B40C8091850C20
:107C1000981709F440C08091920C992787FD9095A0
:107C20002817390731F49091B40C8091A70C98175C
:107C300091F18091A90C992787FD90952817390714
:107C400031F49091B40C8091A60C981721F1809199
:107C5000B30C992787FD90952817390731F4909137
:107C6000B40C8091970C9817B1F06C30A4F46D5F50
:107C70006093B00C63508091B40C42E150E00E94DC
:107C8000A42A8091B40C6091B00C63508F5F42E1E4
:107C900050E00E94A42A8091AD0C813009F070C19F
:107CA0004091850C80918A0C84170CF055C0242FCC
:107CB000332727FD3095235030408091B40C99270D
:107CC00087FD90952817390739F490917F0C8091A2
:107CD000B00C981709F440C08091A70C992787FD34
:107CE00090952817390731F490917F0C8091920C70
:107CF000981791F18091A60C992787FD90952817E8
:107D0000390731F490917F0C8091A90C981721F1DB
:107D10008091970C992787FD90952817390731F4A2
:107D200090917F0C8091B30C9817B1F04830A4F07B
:107D300043504093850C4D5F842F60917F0C42E14E
:107D400050E00E94A42A8091850C8C5F60917F0C8A
:107D500042E150E00E94A42A4091850C80918A0C57
:107D600048170CF055C0242F332727FD30952D5F81
:107D70003F4F8091B40C992787FD909528173907BC
:107D800039F490917F0C8091B00C981709F440C0A1
:107D90008091A70C992787FD90952817390731F412
:107DA00090917F0C8091920C981791F18091A60C84
:107DB000992787FD90952817390731F490917F0C0A
:107DC0008091A90C981721F18091970C992787FD34
:107DD00090952817390731F490917F0C8091B30C5E
:107DE0009817B1F04032A4F44D5F4093850C435096
:107DF000842F60917F0C42E150E00E94A42A809180
:107E0000850C825060917F0C42E150E00E94A42AD0
:107E100060917F0C8091A20C86170CF055C0262F24
:107E2000332727FD3095235030408091B00C99279F
:107E300087FD90952817390739F49091850C80912A
:107E4000B40C981709F440C08091920C992787FDD3
:107E500090952817390731F49091850C8091A70CE3
:107E6000981791F18091A90C992787FD9095281773
:107E7000390731F49091850C8091A60C981721F167
:107E80008091B30C992787FD90952817390731F415
:107E90009091850C8091970C9817B1F06930A4F0FF
:107EA000635060937F0C6D5F8091850C42E150E0E0
:107EB0000E94A42A8091850C60917F0C6D5F8F5F7A
:107EC00042E150E00E94A42A60917F0C8091A20CB4
:107ED00068170CF055C0262F332727FD30952D5FEE
:107EE0003F4F8091B00C992787FD9095281739074F
:107EF00039F49091850C8091B40C981709F440C026
:107F00008091920C992787FD90952817390731F4B5
:107F10009091850C8091A70C981791F18091A90CF4
:107F2000992787FD90952817390731F49091850C92
:107F30008091A60C981721F18091B30C992787FDA9
:107F400090952817390731F49091850C8091970C02
:107F50009817B1F06C30A4F46D5F60937F0C6350A0
:107F60008091850C42E150E00E94A42A8091850C0A
:107F700060917F0C63508F5F42E150E00E94A42A21
:107F80008091B20C813009F070C14091A70C8091B2
:107F90008A0C84170CF055C0242F332727FD309509
:107FA000235030408091B40C992787FD9095281775
:107FB000390739F49091920C8091B00C981709F41C
:107FC00040C08091850C992787FD90952817390727
:107FD00031F49091920C80917F0C981791F18091DF
:107FE000A60C992787FD90952817390731F49091B1
:107FF000920C8091A90C981721F18091970C9927E8
:1080000087FD90952817390731F49091920C809153
:10801000B30C9817B1F04230A4F043504093A70C32
:108020004D5F842F6091920C42E150E00E94A42A9F
:108030008091A70C8C5F6091920C42E150E00E940D
:10804000A42A4091A70C80918A0C48170CF055C0C7
:10805000242F332727FD30952D5F3F4F8091B40C9F
:10806000992787FD90952817390739F49091920C3C
:108070008091B00C981709F440C08091850C992725
:1080800087FD90952817390731F49091920C8091D3
:108090007F0C981791F18091A60C992787FD9095F8
:1080A0002817390731F49091920C8091A90C9817F8
:1080B00021F18091970C992787FD90952817390712
:1080C00031F49091920C8091B30C9817B1F0433138
:1080D000A4F44D5F4093A70C4350842F6091920C01
:1080E00042E150E00E94A42A8091A70C8250609146
:1080F000920C42E150E00E94A42A6091920C80917F
:10810000A20C86170CF055C0262F332727FD30957B
:10811000235030408091B00C992787FD9095281707
:10812000390739F49091A70C8091B40C981709F491
:1081300040C080917F0C992787FD909528173907BB
:1081400031F49091A70C8091850C981791F1809152
:10815000A90C992787FD90952817390731F490913C
:10816000A70C8091A60C981721F18091B30C992748
:1081700087FD90952817390731F49091A70C8091CD
:10818000970C9817B1F01616A4F463506093920CF4
:108190006D5F8091A70C42E150E00E94A42A80917B
:1081A000A70C6091920C6D5F8F5F42E150E00E94DE
:1081B000A42A6091920C8091A20C68170CF055C013
:1081C000262F332727FD30952D5F3F4F8091B00C30
:1081D000992787FD90952817390739F49091A70CB6
:1081E0008091B40C981709F440C080917F0C9927B6
:1081F00087FD90952817390731F49091A70C80914D
:10820000850C981791F18091A90C992787FD90957D
:108210002817390731F49091A70C8091A60C981774
:1082200021F18091B30C992787FD90952817390784
:1082300031F49091A70C8091970C9817B1F06430AD
:10824000A4F46D5F6093920C63508091A70C42E19F
:1082500050E00E94A42A8091A70C6091920C635078
:108260008F5F42E150E00E94A42A8091A40C8130EB
:1082700009F070C14091A60C80918A0C84170CF013
:1082800055C0242F332727FD30952350304080914F
:10829000B40C992787FD90952817390739F49091E8
:1082A000A90C8091B00C981709F440C08091850CFE
:1082B000992787FD90952817390731F49091A90CDB
:1082C00080917F0C981791F18091A70C992787FDD9
:1082D00090952817390731F49091A90C8091920C50
:1082E000981721F18091970C992787FD9095281771
:1082F000390731F49091A90C8091B30C9817B1F023
:108300004230A4F043504093A60C4D5F842F6091FF
:10831000A90C42E150E00E94A42A8091A60C8C5F37
:108320006091A90C42E150E00E94A42A4091A60C61
:1083300080918A0C48170CF055C0242F332727FD55
:1083400030952D5F3F4F8091B40C992787FD909514
:108350002817390739F49091A90C8091B00C98171F
:1083600009F440C08091850C992787FD90952817C6
:10837000390731F49091A90C80917F0C981791F1F5
:108380008091A70C992787FD90952817390731F41C
:108390009091A90C8091920C981721F18091970CE3
:1083A000992787FD90952817390731F49091A90CEA
:1083B0008091B30C9817B1F04331A4F44D5F409312
:1083C000A60C4350842F6091A90C42E150E00E941A
:1083D000A42A8091A60C82506091A90C42E150E041
:1083E0000E94A42A6091A90C8091A20C86170CF01F
:1083F00055C0262F332727FD3095235030408091DC
:10840000B00C992787FD90952817390739F490917A
:10841000A60C8091B40C981709F440C080917F0C91
:10842000992787FD90952817390731F49091A60C6C
:108430008091850C981791F18091920C992787FD76
:1084400090952817390731F49091A60C8091A70CCC
:10845000981721F18091B30C992787FD90952817E3
:10846000390731F49091A60C8091970C9817B1F0D0
:108470001616A4F463506093A90C6D5F8091A60C4E
:1084800042E150E00E94A42A8091A60C6091A90CC0
:108490006D5F8F5F42E150E00E94A42A6091A90CB9
:1084A0008091A20C68170CF055C0262F332727FDAA
:1084B00030952D5F3F4F8091B00C992787FD9095A7
:1084C0002817390739F49091A60C8091B40C9817AD
:1084D00009F440C080917F0C992787FD909528175B
:1084E000390731F49091A60C8091850C981791F181
:1084F0008091920C992787FD90952817390731F4C0
:108500009091A60C8091A70C981721F18091B30C43
:10851000992787FD90952817390731F49091A60C7B
:108520008091970C9817B1F06430A4F46D5F60935C
:10853000A90C63508091A60C42E150E00E94A42A4D
:108540008091A60C6091A90C63508F5F42E150E0CE
:108550000E94A42A8091840C813009F070C140915E
:10856000970C80918A0C84170CF055C0242F332768
:1085700027FD3095235030408091B40C992787FD1A
:1085800090952817390739F49091B30C8091B00C6D
:10859000981709F440C08091850C992787FD909524
:1085A0002817390731F49091B30C80917F0C9817FC
:1085B00091F18091A70C992787FD9095281739078D
:1085C00031F49091B30C8091920C981721F1809125
:1085D000A60C992787FD90952817390731F49091BB
:1085E000B30C8091A90C9817B1F04230A4F043501D
:1085F0004093970C4D5F842F6091B30C42E150E0A3
:108600000E94A42A8091970C8C5F6091B30C42E188
:1086100050E00E94A42A4091970C80918A0C481740
:108620000CF055C0242F332727FD30952D5F3F4F89
:108630008091B40C992787FD90952817390739F454
:108640009091B30C8091B00C981709F440C08091C0
:10865000850C992787FD90952817390731F490915B
:10866000B30C80917F0C981791F18091A70C9927FA
:1086700087FD90952817390731F49091B30C8091BC
:10868000920C981721F18091A60C992787FD90955F
:108690002817390731F49091B30C8091A90C9817E1
:1086A000B1F04331A4F44D5F4093970C4350842FB5
:1086B0006091B30C42E150E00E94A42A8091970C93
:1086C00082506091B30C42E150E00E94A42A609174
:1086D000B30C8091A20C86170CF055C0262F3327BF
:1086E00027FD3095235030408091B00C992787FDAD
:1086F00090952817390739F49091970C8091B40C14
:10870000981709F440C080917F0C992787FD9095B8
:108710002817390731F49091970C8091850C9817A0
:1087200091F18091920C992787FD90952817390730
:1087300031F49091970C8091A70C981721F18091BA
:10874000A90C992787FD90952817390731F4909146
:10875000970C8091A60C9817B1F01616A4F46350EC
:108760006093B30C6D5F8091970C42E150E00E94E2
:10877000A42A8091970C6091B30C6D5F8F5F42E1EA
:1087800050E00E94A42A6091B30C8091A20C68175B
:108790000CF055C0262F332727FD30952D5F3F4F16
:1087A0008091B00C992787FD90952817390739F4E7
:1087B0009091970C8091B40C981709F440C0809167
:1087C0007F0C992787FD90952817390731F49091F0
:1087D000970C8091850C981791F18091920C9927B4
:1087E00087FD90952817390731F49091970C809167
:1087F000A70C981721F18091A90C992787FD9095D6
:108800002817390731F49091970C8091A60C98178E
:10881000B1F06430A4F46D5F6093B30C6350809149
:10882000970C42E150E00E94A42A8091970C60913D
:10883000B30C63508F5F42E150E00E94A42A089578
:10884000CF93DF9380918B0C882329F485E160E935
:1088500041E00E94E72EC0E0D0E080918A0C609158
:10886000A20C42E150E00E94A42A80918A0C8F5F02
:108870006091A20C42E150E00E94A42A83E090E0C3
:108880000E94523680918A0C6091A20C4FEE50E00B
:108890000E94A42A80918A0C8F5F6091A20C40EF05
:1088A00050E00E94A42A82E090E00E945236219675
:1088B000C630D10591F68091A30C8430D9F5809112
:1088C000AA0C9091AB0C18161906A4F580918B0C8C
:1088D000882329F489E160E941E00E94E72E8AE0DB
:1088E00090E06BE070E041E059E00E94333680E0B8
:1088F0000E94D22A83FFFBCF8091820C9091830C3F
:10890000CC970CF094C08091AA0C9091AB0C059779
:108910000CF48DC08091A50C882331F08091980CC7
:108920009091990C02967FC080918E0C90918F0C43
:1089300002966FC08091A30C833079F48091AA0CC9
:108940009091AB0C1816190644F488E090E06BE0A7
:1089500070E046E159E00E94333680E00E94D22A5E
:1089600083FF16C08091A30C8F5F8093A30C80912E
:10897000AA0C9091AB0C892B49F481E08093A30C55
:108980008AE090E09093AB0C8093AA0C80E050C0FA
:1089900090FFD0CF8091A30C833061F684E0809368
:1089A000A30C8091AA0C9091AB0C892B49F481E027
:1089B0008093A30C8AE090E09093AB0C8093AA0C78
:1089C0008091820C9091830CC3978CF10E94274771
:1089D0006CE470E02091820C3091830C621B730B6D
:1089E0000E946A468093A80C8150893000F58091DE
:1089F0008B0C882329F489E160E941E00E94E72E8D
:108A00008091A50C882351F080918E0C90918F0C51
:108A1000039690938F0C80938E0C09C08091980CD4
:108A20009091990C03969093990C8093980C81E007
:108A30000E947838DF91CF91089580918B0C882324
:108A400029F489E160E941E00E94E72E8091AC0CB5
:108A50008F5F8093AC0C813041F488E090E06BE054
:108A600070E04FE259E00E9433368091AC0C8230C6
:108A700041F488E090E06BE070E044E459E00E944B
:108A800033368091AC0C833041F488E090E06BE0A9
:108A900070E049E559E00E9433368091AC0C843097
:108AA00011F40E947E4588E090E06EE070E041E0C5
:108AB00059E00E94333680E00E94D22A83FFFBCF28
:108AC0008091AE0C9091AF0C892BB9F48091A50CDC
:108AD000813051F488E790E09093AF0C8093AE0C16
:108AE00081E00E947838089588E790E09093AF0C79
:108AF0008093AE0C82E00E94783808950E947E2A0E
:108B000080918B0C882329F489E160E941E00E947F
:108B1000E72E8AE090E062E070E04EE659E00E94C5
:108B2000333682E090E064E170E040EA59E00E9470
:108B3000333620918E0C30918F0C8091980C90914F
:108B4000990C8217930784F482E090E066E070E06D
:108B500048ED58E00E94333682E090E067E070E034
:108B600043E859E00E9433362091980C3091990CDB
:108B700080918E0C90918F0C8217930784F482E081
:108B800090E066E070E04DED58E00E94333682E000
:108B900090E067E070E043E859E00E94333640918E
:108BA0008E0C50918F0C8091980C9091990C841799
:108BB0009507C4F48DE090E067E070E020E00E944B
:108BC000013680E190E067E070E04DE859E00E94F6
:108BD000333685E190E067E070E04091980C20E04A
:108BE0000E9401364091980C5091990C80918E0C06
:108BF00090918F0C84179507C4F48DE090E067E0A6
:108C000070E020E00E94013680E190E067E070E0D3
:108C10004DE859E00E94333685E190E067E070E06E
:108C200040918E0C20E00E94013620918E0C3091F4
:108C30008F0C8091980C9091990C2817390711F599
:108C400082E090E066E070E040E959E00E9433364F
:108C500082E090E067E070E040918E0C20E00E949E
:108C6000013685E090E067E070E04DE859E00E9451
:108C700033368AE090E067E070E04091980C20E0A5
:108C80000E94013680E00E94D22A83FFFBCF0C9421
:108C900000000895991B79E004C0991F961708F009
:108CA000961B881F7A95C9F780950895AA1BBB1B50
:108CB00051E107C0AA1FBB1FA617B70710F0A61BDC
:108CC000B70B881F991F5A95A9F780959095BC01FD
:108CD000CD01089597FB092E07260AD077FD04D011
:108CE000E5DF06D000201AF4709561957F4F089556
:108CF000F6F7909581959F4F0895A1E21A2EAA1B31
:108D0000BB1BFD010DC0AA1FBB1FEE1FFF1FA2173B
:108D1000B307E407F50720F0A21BB30BE40BF50B38
:108D2000661F771F881F991F1A9469F760957095C1
:108D3000809590959B01AC01BD01CF0108952F92C4
:108D40003F924F925F926F927F928F929F92AF92DB
:108D5000BF92CF92DF92EF92FF920F931F93CF9328
:108D6000DF93CDB7DEB7CA1BDB0B0FB6F894DEBFBF
:108D70000FBECDBF09942A88398848885F846E84E5
:108D80007D848C849B84AA84B984C884DF80EE802F
:108D9000FD800C811B81AA81B981CE0FD11D0FB638
:108DA000F894DEBF0FBECDBFED010895A0E0B0E0A6
:108DB000ECEDF6E40C94A746EC01A880B980CA80DB
:108DC000DB80A114B104C104D10441F484E2A82ED3
:108DD00089EDB82E8BE5C82E87E0D82EC601B501E7
:108DE0002DE133EF41E050E00E94564727EA31E49D
:108DF00040E050E00E9437477B018C01C601B5017D
:108E00002DE133EF41E050E00E945647CA01B9011D
:108E10002CEE34EF4FEF5FEF0E9437476E0D7F1D52
:108E2000801F911F97FF04C06150704080409048A0
:108E3000688379838A839B839B013F77C901CDB780
:108E4000DEB7EAE00C94C3460E94D646089580E05F
:108E500091E00E94D6460895A0E0B0E08093000122
:108E600090930101A0930201B09303010895629FC2
:108E7000D001739FF001829FE00DF11D649FE00D12
:108E8000F11D929FF00D839FF00D749FF00D659F73
:108E9000F00D9927729FB00DE11DF91F639FB00D72
:108EA000E11DF91FBD01CF011124089597FB092E83
:108EB00005260ED057FD04D020DF0AD0001C38F460
:108EC00050954095309521953F4F4F4F5F4F0895F6
:108ED000F6F790958095709561957F4F8F4F9F4FD6
:068EE0000895F894FFCF95
:048EE6000100000087
:00000001FF
